:200000000C9494030C9464240C9491240C94BC030C94BC030C94BC030C94BC030C949A294D
:200020000C94BC030C94BC030C94BC030C94BC030C94BC030C94BC030C94BC030C94BC03C8
:200040000C94BE240C94BC030C9499260C94EB260C94BC030C94BC030C94BC030C94BC0333
:200060000C949D220C94BC03B610B210B210B610B210B210B210B210B210B210B210B210A2
:20008000B210B210B210B210B210B210B210B210B210B2105B1082109A10B2109D10B210F4
:2000A0008B107F10851088107610A3107C1094107910581037103A103D10401043104610B8
:2000C00049104C104F1052108E109110A3105510A610B210A010E90FEC0FEF0FF20FF50F35
:2000E000F80FFB0FFE0F0110041007100A100D1010101310161019101C101F10221025101B
:2001000028102B102E1031103410B210B210B210B2109710B210B210B210B210B210B2106E
:20012000B210B210B210B210B210B210B210B210B210B210B210B210B210B210B210B2109F
:20014000B210B210B210B210B210B210A910581A871A751A6F1A1D1D1D1D1D1D1D1D1D1D0D
:200160001D1D1D1D1D1D1D1D411A1D1D1D1D1D1D251A2F1AD91A1D1D1D1D1D1D1D1D1D1DF1
:200180001D1D1D1D1D1D1D1D1D1D1D1D1D1D1D1D1D1D1D1D1D1D1D1D1D1D1D1D1D1D1D1DBF
:2001A0001D1D1D1D1D1D1D1D1D1D1D1D1D1D1D1D1D1D1D1D1D1D1D1D1D1D1D1D1D1D1D1D9F
:2001C0001D1D1D1D1D1D1D1D1D1D1D1D1D1D1D1D1D1D1D1D1D1D1D1D1D1D1D1D1D1D1D1D7F
:2001E0001D1D1D1D1D1D1D1D1D1D1D1D1D1D1D1D1D1D1D1D1D1D1D1D1D1D1D1D1D1D1D1D5F
:200200001D1D1D1D1D1D1D1D1D1D1D1D1D1D1D1D1D1D1D1D1D1D1D1D1D1D1D1D1D1D1D1D3E
:200220001D1D1D1D1D1D1D1D1D1D1D1D1D1D1D1D1D1D1D1D1D1D1D1D1D1D1D1DD01A241B69
:200240007D1A9C1A9E1AA21AA41AA61AA81AAA1AAC1AAE1AB01AB21AB41A981A0A1B0C1BE9
:200260000E1B101B121B141B161B181B1A1B1C1B1E1B201B1D1D301B331B601D1D1D1D1DC6
:200280001D1D6E1B781B1D1D821B8C1B1D1DAD1BC01BCD1B1D1D1D1D1D1D601DF01B1C1C57
:2002A0001D1D1D1D1D1D1D1D4E1C741C1D1D941C1D1D1D1DE71CBB1CD11C601D601D601DC0
:2002C000601D1D1D1D1D1D1D1D1D1D1D1D1DB61AB81ABA1ABC1ABE1AC01AC21AC41AC61AAD
:2002E000C81ACA1ACC1A3FE019C063019C3FE03030FFC3330CCC1CE03FF0C0C3030C0C3015
:20030000303030FFC3030C0C1FE03FF0CCC3330C0C30303FF00CC033000C00303FF0C0C3EC
:20032000030CCC3F303FF00C003000C03FF000000003FF000000003C00C003000C003FF0DD
:200340003FF00C0070033038E03FF0C003000C0030003FF001800C00183FF03FF00380388C
:2003600003803FF03FF0C0C3030C0C3FF03030FFC33300CC03F03FF0C0C3C30FFCF0003F0C
:20038000F00CC03303CC39E031E0CCC3330CCC1E30003000C3FF000C00303FF0C003000C61
:2003A000003FF03FF0700070007000701FF0C001F00C001FF03870330078033038700070A6
:2003C0000703F0007000703830F8C3330C7C30701FE0C0C3030C0C1FE000000300060FFC15
:2003E00000003860F0C3330C783000C00300C6330CFC1E0007F81800600FFC06003000C071
:20040000031F86660F181FF0CC6318CC601F00703070C073007C00703CF19E663199E63CBA
:20042000F003E318C6630C0C1FE003000C01FE00C0030003000C003000C00300003000CEBD
:2004400073007C00007000700070007000703800E00000000000000C01F000000000000068
:200460000038038000000000000CC03300CC03300CC070387380780000000000000000786C
:200480000738703800007381CE000000000000000000000000004E6F2073657269616C2036
:2004A000666561747572657320656E61626C65642E2E2E0000970093918F909A0098969432
:2004C00092097E00000000000051210000005A5341574000004358444524230000205646E5
:2004E00054522500004E424847595E0000004D4A55262A00003C4B494F292800003E3F4CE6
:200500003A505F00000022007B2B000000000D7D007C00000000000000009D000031003422
:2005200037000000302E323536381B00992B332D2A39A0000000009500C400C0BEBCBDC7F8
:2005400000C5C3C1BF097E0000000000005121000000BB53A2B84000004358A5A6242300C5
:2005600000205646B552250000AFA3A9A8595E000000AE4AB6262A00003C4BAAB029280009
:20058000003E3F4C3A505F00000022007B2B000000000D7D007C00000000000000009D003E
:2005A0000031003437000000302E323536381B00992B332D2A39A0000000009500D000CCF9
:2005C000CAC8C9D300D1CFCDCB097E0000000000005121000000BB53A2B84000004358A5D4
:2005E000A624230000205646B552250000AFA3A9A8595E000000AE4AB6262A00003C4BAA9D
:20060000B0292800003E3F4C3A505F00000022007B2B000000000D7D007C00000000000059
:2006200000009D000031003437000000302E323536381B00D22B332D2A39A000000000CE05
:20064000008A00868482838D008B898785096000009E00000071310000007A7361773200B4
:2006600000637864653433000020766674723500006E62686779360000006D6A753738004F
:20068000002C6B696F303900002E2F6C3B702D00000027005B3D000000000D5D005C00005C
:2006A0000000000000007F000031003437000000302E323536381B008C2B332D2A398E00C9
:2006C0000000008800000000240027002A0000000000250028002B0000000000230026005C
:2006E000290004040404040404040202020202020303030303030102040810204080010291
:20070000040810200102040810200000000700020100000304060000000000000000020045
:20072000FF060A225A28F80611241FBECFEFD8E0DEBFCDBF13E0A0E0B1E0EEE6F6E602C0E1
:2007400005900D92A639B107D9F716E0A6E9B3E001C01D92AF37B107E1F717E0C6E2D7E0AA
:2007600004C02297FE010E942633C032D107C9F70E945F2E0C942A330C940000FB01DC01D3
:2007800002C001900D9241505040D8F70895FB01DC0101900D920020E1F70895FB019F01A0
:2007A000E8944230C4F04532B4F44A3029F497FB1EF4909581959F4F642F77270E94C0324F
:2007C000805D8A330CF0895D8193CB010097A1F716F45DE251931082C9010C940504FB0160
:2007E0009F01423074F0453264F4642F77270E94C032805D8A330CF0895D8193CB010097FC
:20080000A1F71082C9010C940504DC01FC01672F71917723E1F7329704C07C916D937083CA
:200820006291AE17BF07C8F30895982F8C30D0F4E0918B04E63940F4EF5FE0938B04F0E028
:20084000EC50FC4F87E18083E0918B04E63938F4EF5FE0938B04F0E0EC50FC4F90838FEF23
:2008600080935C030895982F813019F08230B1F40BC08DE08093A4038BE0809348039093B3
:20088000A5039093C20308951092A4038CE0809348039093A50381E08093C20308956F33D5
:2008A00028E0720720E0820720E0920709F4B4C1603428E0720720E0820720E092070CF0F0
:2008C000BCC06A3771058105910509F4E7C16B377105810591050CF04FC06C3071058105ED
:2008E000910509F49CC16D30710581059105FCF4623071058105910509F4C7C16330710537
:20090000810591053CF4613071058105910509F007C28EC1693071058105910509F4F7C177
:200920006B3071058105910509F0FAC18DC16F3671058105910509F4A5C16037710581055B
:2009400091056CF4653171058105910509F48BC1663171058105910509F0E2C181C1603792
:2009600071058105910509F493C1693771058105910509F0D5C183C1673524E0720720E076
:20098000820720E0920709F45CC1683524E0720720E0820720E09207FCF4643D7105810552
:2009A000910509F457C1653D7105810591053CF4633D71058105910509F0B2C136C16D3DE9
:2009C00071058105910509F439C16E3D71058105910509F0A5C14AC16B3B24E0720720E0C4
:2009E000820720E0920709F438C16C3B24E0720720E0820720E0920784F4683524E0720707
:200A000020E0820720E0920709F445C1615674408040904009F084C10EC1653C24E072078B
:200A200020E0820720E0920709F423C1665C74408040904009F074C10AC16E3B2FE2720781
:200A400020E0820720E0920709F437C16F3B2FE2720720E0820720E092070CF06AC0643A65
:200A600028E0720720E0820720E0920709F404C1653A28E0720720E0820720E0920744F596
:200A8000693428E0720720E0820720E0920709F4C9C06A3428E0720720E0820720E092074F
:200AA0003CF4605478408040904009F039C1F9C06A3428E0720720E0820720E0920709F420
:200AC000F3C0635A78408040904009F029C1EFC062372BE2720720E0820720E0920709F48E
:200AE000F2C063372BE2720720E0820720E0920784F467362BE2720720E0820720E0920745
:200B000009F4E7C068567B428040904009F008C1DDC0663D2BE2720720E0820720E092077C
:200B200009F4CEC069557F428040904009F0F8C0F4C06D3C26E5720720E0820720E0920767
:200B400009F4D3C06E3C26E5720720E0820720E092078CF5613822E5720720E0820720E092
:200B6000920709F4C8C0623822E5720720E0820720E0920784F4673722E5720720E08207FC
:200B800020E0920709F4A8C0685772458040904009F0C6C0BFC06F3526E5720720E08207A2
:200BA00020E0920709F49BC0635C76458040904009F0B6C097C0623C2FE5720723E08207BD
:200BC00020E0920709F49DC0633C2FE5720723E0820720E0920784F46E3C26E5720720E02B
:200BE000820720E0920709F465C06355764B8140904009F095C07CC06E3024E6720723E0F9
:200C0000820720E0920709F47FC06C5E76438042904009F085C072C022E430E083C021E493
:200C200030E080C023E430E07DC024E430E07AC025E430E077C026E430E074C027E430E005
:200C400071C028E430E06EC029E430E06BC02AE430E068C02BE430E065C02CE430E062C005
:200C60002DE430E05FC02EE430E05CC02FE430E059C020E530E056C021E530E053C022E55F
:200C800030E050C023E530E04DC024E530E04AC025E530E047C026E530E044C027E530E090
:200CA00041C028E530E03EC029E530E03BC02AE530E038C020E330E035C021E330E032C0DA
:200CC00022E330E02FC023E330E02CC024E330E029C025E330E026C026E330E023C027E30A
:200CE00030E020C028E330E01DC029E330E01AC02FE330E017C02FE230E014C02AE230E00C
:200D000011C02CE230E00EC02CE530E00BC020E230E008C02DE330E005C02BE230E002C08C
:200D20002EEF30E0C90108951092C10381E08093BC038AE190E090939703809396038AE0D8
:200D40008093EE0388E592E090939C0380939B0388EB9BE09093A8038093A70381E280934E
:200D6000AB038CE291E090939E0380939D0387E08093A00382E38093A60381E00E943304F7
:200D80000895CF92EF920F938130910501F56F5F7F4F51F589ED93E060E071E00E94352D95
:200DA0008FED93E060E071E00E94352D83E994E00E94651F84E994E060E14AE026E007E070
:200DC00058E0E52E39E0C32E0E94A1210DC0892B59F46F5F7F4F41F48FED93E00E94522EAA
:200DE00089ED93E00E94522E0F91EF90CF90089580E090E06FEF7FEF0E94C106089581E0CA
:200E000090E06FEF7FEF0E94C1060895CF92DF92EF92FF920F931F93CF93DF939C01FC01EA
:200E2000EE51F94FE4918E2F90E0880F991FFC01E253F94F05911491FC01EC53F94FE5908C
:200E4000F4902A50394FF901D490FC01E852F94FC591D491F8018081CD2CC0948C2180837D
:200E6000F70180818D29808361E070E080E090E00E941425F894F70180818C218083F80156
:200E800080818D29808388812D2D30E090E082239323892B11F090E081C0888190E08223D6
:200EA0009323892B11F091E079C0888190E082239323892B11F092E071C0888190E08223D3
:200EC0009323892B11F093E069C0888190E082239323892B11F094E061C0888190E08223CF
:200EE0009323892B11F095E059C0888190E082239323892B11F096E051C0888190E08223CB
:200F00009323892B11F097E049C0888190E082239323892B11F098E041C0888190E08223C6
:200F20009323892B11F099E039C0888190E082239323892B11F09AE031C0888190E08223C2
:200F40009323892B11F09BE029C0888190E082239323892B11F09CE021C0888190E08223BE
:200F60009323892B11F09DE019C0888190E082239323892B11F09EE011C0888190E08223BA
:200F80009323892B11F09FE009C0888190E082239323892B11F491E101C090E17894F80168
:200FA00080818C218083F70180818D298083892FDF91CF911F910F91FF90EF90DF90CF901A
:200FC00008950E94060720E030E0833010F421E030E0C901089582E090E00E94E107892B76
:200FE00049F085E090E00E94E107892B19F481E080939903089580919803882311F082E031
:2010000001C085E090E00E94E107882341F481E08093BE038FEF80935C031092B9030895B0
:2010200080919803882311F085E001C082E090E00E94E107882371F481E08093BD031092F0
:20104000B90380915C038F3F29F08FEF80935C0310928B0408950E9410080E94FB07809150
:201060009903853009F072C09091CC03992309F05EC08091B104823031F1833030F4882315
:20108000F1F1813009F062C006C0833081F0843009F05CC024C08091BE039091BD038823AD
:2010A000D9F09923E1F184E08093B10420C08091BD039091BE03882319F0992341F141C077
:2010C0009923D1F02CC08091BD039091BE03882319F09923E1F027C09923C1F50DC080917C
:2010E000BE039091BD03882329F09923C1F01092BD030895992359F41092B1040895909100
:20110000BD03992331F08091BE03882311F481E007C08091BE038823C9F0992321F482E01F
:201120008093B104089583E08093B1040AC08091BD03882359F08091BE03882339F0913029
:2011400019F41092BE0308951092BD0308951092BA031092980382E08093990381E0809362
:201160009A031092BB036AEF70E080E090E00E94142508958091C703882349F08091A4030A
:20118000882319F060E00E94F1251092C703089581E161E00E94F125089582E060E00E945E
:2011A000B22582E061E00E94F12585E060E00E94B22585E061E00E94F1258BE061E00E9433
:2011C000B2258BE060E00E94F1258CE061E00E94B2258CE060E00E94F1258DE061E00E94FB
:2011E000B2258DE060E00E94F12584E061E00E94B22584E060E00E94F125089581E068ECE7
:2012000078E042E050E00E94412481E160E00E94F12581E161E00E94B22568EC70E080E0A3
:2012200090E00E94142581E163E00E94661F089583E496E09093AA048093A9044091F003C8
:201240005091F1036091F2037091F3030E94262708952F923F924F925F926F927F928F92B9
:201260009F92AF92BF92CF92DF92EF92FF920F931F93DF93CF930F92CDB7DEB73B014C015C
:2012800019012A01E98220E030E040E050E00E94EB3018160CF09DC08091C803882331F44E
:2012A00080EB94E0B8010E94D4320CC08091550390E028EE33E0829FB001839F700D929F7E
:2012C000700D1124882777FD8095982F0E948A317B018C010E9406255B016C01C201B101EC
:2012E0000E945731A60EB71EC81ED91EC801B701A40193010E943E320E945731A60EB71EDF
:20130000C81ED91E11E036C0833071F482E090E00E94E107892B41F485E090E00E94E1074D
:20132000892B11F41093CD038091C003813019F40E94FB0704C0823011F40E94100889810C
:201340008823C1F482E090E00E94E107892B71F085E090E00E94E107892B41F08091BD03A7
:20136000882321F48091BE03882321F08091BA03882379F10E9406256A157B058C059D053D
:2013800020F50E940625693C710581059105E8F080919903853009F0B7CFD1CF8091CD03FA
:2013A0008823B9F082E090E00E94E107019789F485E090E00E94E107019759F41092CD03B2
:2013C0001092BD031092BE0304C080919903833029F30F90CF91DF911F910F91FF90EF903B
:2013E000DF90CF90BF90AF909F908F907F906F905F904F903F902F9008958091C1038823BC
:2014000059F00E9406256093C3037093C4038093C5039093C60308958091C703882309F44C
:201420004AC08091B903882309F045C080915903813009F50E9406252091C3033091C40344
:201440004091C5035091C603621B730B840B950BE091A503F0E0EE0FFF1FE95BFC4F2081EB
:20146000318140E050E0621773078407950718F10E94BA0808950E9406252091C303309141
:20148000C4034091C5035091C603621B730B840B950BE091A503F0E0EE0FFF1FE95BFC4F85
:2014A0002081318140E050E0261737074807590710F40E94BA0808958091C7038823B9F427
:2014C0008091A403882381F061E00E94F125E091A503F0E0EE0FFF1FE555FC4F60817181E3
:2014E00080E090E00E94142581E08093C7030E9406256093C3037093C4038093C5039093B5
:20150000C603089580915C038C3008F042C00E94062520918E0430918F0440919004509195
:201520009104621B730B840B950B2091A7033091A80340E050E0261737074807590748F56E
:20154000E0918B04E63940F4EF5FE0938B04F0E0EC50FC4F87E1808380915C03E0918B04B6
:20156000E63968F48F3741F0EF5FE0938B04F0E0EC50FC4F808303C0E150E0938B040E94B7
:20158000062560938E0470938F04809390049093910480915C038F3F41F410928E0410925D
:2015A0008F0410929004109291040895CF93DF93CEE1D0E08DEA95E0BE014FEF0E94352477
:2015C000CE5ADF4F83E0C63FD807A1F7DF91CF9108950F931F93CF93DF93892B49F08DEADD
:2015E00095E060E070E043E10E9435240E94D60AC6E9D3E061E070E08B010F5F1F4F499110
:201600008DEA95E00E943524B80108311105A1F71092C203DF91CF911F910F91089580910E
:20162000C203882309F10E9406252091CE033091CF034091D0035091D103621B730B840B7B
:20164000950B615375478040904070F080E090E00E94E90A0E9406256093CE037093CF03BF
:201660008093D0039093D10308950F931F93CF93DF938DEA95E060E070E00E942E248331A4
:2016800019F021E030E018C0C6E9D3E061E070E08B010F5F1F4F8DEA95E00E942E24899301
:2016A000B80108311105A1F78091A5030E9433041092C20320E030E0C901DF91CF911F9137
:2016C0000F91089517C0E091A904F091AA04A081B18116962D913C911797CF01F901099509
:2016E0008093EF038091A9049091AA0466E974E00E942F29E091A904F091AA04A081B1811B
:2017000014962D913C911597CF01F901099518161906CCF2089584E06CED75E028EC30E0A2
:2017200040E050E00E94F629089584E06CED75E020E030E040E050E00E94F62964E670E02E
:2017400080E090E00E94142584E060E971E020E030E040E050E00E94F62964E670E080E0C5
:2017600090E00E94142584E00E948329089582E090E00E94E107892B99F485E090E00E94BB
:20178000E107892B69F482E090E00E94E107892BB1F485E090E00E94E107892B81F4F3CF51
:2017A0000E94350B892BB1F081E090E00E94E90A0E94950B0E94950B0E94950B089581E0C8
:2017C00090E00E94E90A0E94950B0E94950B0E94950BE6CF089584E060E971E020E030E0DE
:2017E00040E050E00E94F62964E670E080E090E00E94142584E00E94832908950F931F93F0
:20180000062F2091C103892BC1F1222309F055C08091BC038823B1F01091C7030E945C0AD6
:2018200080914803882319F061E00E94F1256091CB03662339F0112329F470E080E090E0BD
:201840000E94142590919A03913041F08091BA03823021F0923069F4013059F460919B0340
:2018600070919C0384E020E030E040E050E00E94F62981E08093C10320C02223F1F08091F4
:20188000BC03882349F080914803882319F060E00E94F1250E945C0A90919A03913041F0E5
:2018A0008091BA03823021F0923029F4013019F484E00E9483291092C1031F910F91089575
:2018C0008F929F92AF92BF92CF92DF92EF92FF920F931F93982ED0909603C090970382E0E1
:2018E0008093C00381E090E0692D0E94FE0B60919D0370919E0380E090E00E94883120E0A2
:2019000030E048EC52E40E94EF307B018C016091A60370E080E090E00E94883120E030E05E
:2019200048E452E40E94EF309B01AC01C801B7010E943E327B018C016091CA0370E080E031
:2019400090E00E9488319B01AC01C801B7010D2D1C2DE92C0E94290980E090E0692D0E947E
:20196000FE0B6091A60370E080E090E00E94883120E030E048E452E40E94EF3020E030E006
:2019800040E450EC0E943E3220E030E040E850E40E9487307B018C016091CA0370E088274A
:2019A00077FD8095982F0E948A319B01AC015058C801B7010D2D1C2DE92C0E94290981E03B
:2019C000981619F58091A103882309F49EC00E942B089BC08091BD038823B9F48091BE0365
:2019E000882399F4009196031091970360E070E080E090E420E030E040E050E0EE24E394FD
:201A00000E9429098824839401C0882480915A03882309F469C081E0981609F065C02091A5
:201A2000E6033091E7034091E8035091E903DA01C90162E0880F991FAA1FBB1F6A95D1F7E9
:201A4000820F931FA41FB51F0196A11DB11D880F991FAA1FBB1F8093E6039093E703A0935B
:201A6000E803B093E9030E9406250E9488315B016C01609196037091970380E090E00E94C4
:201A800088319B01AC0160E070E086E993E40E94EF307B018C016091580370E0882777FD45
:201AA0008095982F0E948A319B01AC01C801B7010E943E329B01AC01C601B5010E948730F2
:201AC0000E945C316093EA037093EB038093EC039093ED03882041F01092EA031092EB03F9
:201AE0001092EC031092ED030E942B081092C003909259031F910F91FF90EF90DF90CF90DF
:201B0000BF90AF909F908F9008958091A103882309F060CF7ACF8F929F92AF92BF92CF9236
:201B2000DF92EF92FF920F931F93982ED0909603C090970381E08093C00381E090E0692D87
:201B40000E94FE0B6091A60370E080E090E00E94883120E030E048E452E40E94EF307B0116
:201B60008C016091CA0370E080E090E00E9488319B01AC01C801B7010D2D1C2DE92C0E949B
:201B8000290980E090E0692D0E94FE0B6091A60370E080E090E00E94883120E030E048E4B1
:201BA00052EC0E94EF3020E030E040E050E40E9487307B018C016091CA0370E0882777FD2F
:201BC0008095982F0E948A319B01AC015058C801B7010D2D1C2DE92C0E94290981E09816DF
:201BE00019F58091A103882309F494C00E942B0891C08091BD038823B9F48091BE0388235A
:201C000099F4009196031091970360E070E080E090E420E030E040E050E0EE24E3940E94E3
:201C200029098824839401C0882480915A03882309F45FC081E0981609F05BC06091E60310
:201C40007091E7038091E8039091E9032AE030E040E050E00E94A1326F5F7F4F8F4F9F4F49
:201C60006093E6037093E7038093E8039093E9030E9406250E9488315B016C016091960313
:201C80007091970380E090E00E9488319B01AC0160E070E086E993E40E94EF307B018C01F5
:201CA0006091580370E0882777FD8095982F0E948A319B01AC01C801B7010E943E329B01B4
:201CC000AC01C601B5010E9487300E945C316093EA037093EB038093EC039093ED038820C4
:201CE00041F01092EA031092EB031092EC031092ED031092C003909259030E942B081F9109
:201D00000F91FF90EF90DF90CF90BF90AF909F908F9008958091A103882309F06ACF84CFE9
:201D20000F931F93CF93DF938C01C0E0D0E0F801EC0FFD1FE081ED3231F0EE3299F480E0E0
:201D40000E948B0D03C080E00E94600C8091BD03882341F48091BE03882321F42196CC3022
:201D6000D10529F7DF91CF911F910F91089590919903892F8250823018F0953061F54EC086
:201D8000933009F04BC08091CD03882309F446C082E090E00E94E107892B09F43FC085E07C
:201DA00090E00E94E107892BC9F11092CD031092BD031092BE0308951092BD0381E00E9482
:201DC0008B0D8091BE03882371F11092BE0381E00E94600C0895943081F48091BD03882368
:201DE00029F01092BD0381E00E948B0D8091BE03882371F01092BE0308C09130A1F480915D
:201E0000BD03882329F01092BD0381E090E002C080E090E061E00E94FE0B08958091BD031F
:201E2000882379F2C9CF0895882319F081E090E002C080E090E060E00E94FE0B89EB9FE062
:201E40000E946D250895CF92DF92FF920F931F93CF93DF938C01060F111DFF241FC088E0EC
:201E6000F81619F4C230D10574F0C6010C2E02C0959587950A94E2F780FF02C081E001C038
:201E800080E00E94140F2197EFEFCF3FDE0739F7F3940F5F1F4FF9E0FF1639F0C7E0D0E093
:201EA000F8018491C82EDD24DACFDF91CF911F910F91FF90DF90CF9008950F931F93182FBF
:201EC00000E080E00E94140F0F5F0E30D1F7812F81548A3140F469E0169F602D1124695498
:201EE00086EE92E045C0812F80538A3040F469E0169F602D1124605B80ED93E039C01D32E3
:201F0000E1F01E3260F4193231F11A3218F4183241F523C01B3299F01C3219F518C01A33CD
:201F2000F1F01B3328F41E3281F01F32D1F40BC01D3379F01F33A9F404C081E013C080E0B4
:201F400011C082E00FC083E00DC084E00BC085E009C087E007C088E005C089E003C08AE001
:201F600001C08BE069E0869FB00111248AE294E00E94230F10E080E00E94140F1F5F1E304C
:201F8000D1F71F910F910895EF92FF920F931F93982FF62E8A3009F406C18D3009F403C13F
:201FA0008091BB03882309F0FBC0892F992787FD9095A92FB92FFC013A97E337F10508F03C
:201FC000D1C0EC5CFF4FEE0FFF1F0590F491E02D099481E091E0C8C084E091E0C5C089E0DE
:201FE00091E0C2C08EE091E0BFC082E191E0BCC084E191E0B9C089E191E0B6C08DE191E0C1
:20200000B3C082E291E0B0C085E291E0ADC08AE291E0AAC08EE291E0A7C083E391E0A4C0F9
:2020200086E391E0A1C089E391E09EC08DE391E09BC082E491E098C087E491E095C08BE41F
:2020400091E092C08FE491E08FC081E591E08CC085E591E089C08AE591E086C08EE591E039
:2020600083C083E691E080C088E691E07DC08DE691E07AC083E791E077C089E791E074C0A2
:202080008FE791E071C085E891E06EC08BE891E06BC081E991E068C087E991E065C08DE98E
:2020A00091E062C083EA91E05FC089EA91E05CC08FEA91E059C06091A00370E06250704047
:2020C00020915803621B7109882777FD8095982F0E948A31009196031091970320E030E02C
:2020E00040E050E0EE240E94290940C085EB91E03BC08DEB91E038C084EC91E035C08BECA0
:2021000091E032C082ED91E02FC089ED91E02CC08FED91E029C086EE91E026C08CEE91E02E
:2021200023C083EF91E020C080E092E01DC087E092E01AC08EE092E017C085E192E014C034
:202140008DE192E011C08AEF91E00EC084E292E00BC0009196031091970360E070E080E01E
:202160009FE316C08BE292E00E94900E81E0F816D1F06091580370E061507040882777FD98
:202180008095982F0E948A31009196031091970320E030E040E050E0EE240E94290903C098
:2021A000892F0E945D0F1F910F91FF90EF900895DF92EF92FF920F931F93DF93CF93CDB72F
:2021C000DEB72C970FB6F894DEBF0FBECDBF7E010894E11CF11CC70160E071E00E94352DDE
:2021E0008FEF80935C038E01095F1F4F6091560370915703C8014AE00E94802DC701B80122
:202200000E94272EC8010E94522E2D813E812330310560F4E0918B04E63940F4EF5FE0937E
:202220008B04F0E0EC50FC4F80E380832130310561F4E0918B04E63940F4EF5FE0938B04D3
:20224000F0E0EC50FC4F80E38083DD247E010894E11CF11C20C0C701B8010E940C2CC70198
:20226000B8010E940C2CC701B8010E940C2CFC018081E0918B04E63968F48F3741F0EF5FB2
:20228000E0938B04F0E0EC50FC4F808303C0E150E0938B04D3940D2D10E08D819E8108170F
:2022A0001907C8F2C7010E94522E2C960FB6F894DEBF0FBECDBFCF91DF911F910F91FF90A2
:2022C000EF90DF9008950F931F93082F10E084E994E0612F402F0E94B42084E994E062E37C
:2022E00072E00E945F291F5F103189F71F910F91089584E994E00E94E3201092D20308959C
:20230000FF920F931F93CF93DF93EC01F62E8A018091D203823051F08093D70382E080932D
:20232000D20384E994E00E94E32003C0862F0E94631160E170E08C819D81681B790B7695E6
:20234000679584E994E04F2D0E94B42084E994E0BE010E94FD280E940625980140E050E091
:20236000260F371F481F591F2093D3033093D4034093D5035093D603DF91CF911F910F9149
:20238000FF9008950F931F93DF93CF9300D000D000D0CDB7DEB784E994E060E142E020E01C
:2023A0000E94EB208E010F5F1F4FC80164E372E00E94352DC80160E040EA5FE00E948011FA
:2023C000C8010E94522E26960FB6F894DEBF0FBECDBFCF91DF911F910F9108950E94CD08DB
:2023E0000E9494060E94A7080E94B70B0E94EB070E9418090E94FE080E94C2110895CF927A
:20240000DF92EF92FF920F931F93DF93CF93CDB7DEB762970FB6F894DEBF0FBECDBFBC01FB
:20242000809396037093970381E08093C2036E010894C11CD11CC6014AE00E94802D17E00E
:20244000E12EF12CEC0EFD1EC701B6010E94482EC70169E472E00E94E22CBC018E01035FDF
:202460001F4FC8010E943E2EC80160E048EE53E00E948011C8010E94522EC7010E94582E97
:20248000C6010E94522E62960FB6F894DEBF0FBECDBFCF91DF911F910F91FF90EF90DF9077
:2024A000CF9008952F923F924F925F926F927F928F929F92AF92BF92CF92DF92EF92FF92E2
:2024C0000F931F93DF93CF93CDB7DEB7E7970FB6F894DEBF0FBECDBFD82E2DB73EB73EAB2E
:2024E0002DABCDB69EB64DB69FAAE82EFF2482E590E09C01E29EC001E39E900DF29E900DA8
:2025000011249C01225E3F4F3AAB29AB9C0121593F4F3CAB2BAB8DB79EB7825590400FB6BB
:20252000F8949EBF0FBE8DBF2DB63EB60894211C311C5E010894A11CB11CC50160E071E0C0
:202540000E94352D8E01095F1F4FC8016EE472E00E94352D9BE09D1558F40E94EB0BC801C7
:202560000E94522EC5010E94522E8C2D992D07C128E02D1520F0C80160E20E94B52C8E0193
:20258000095F1F4F0894E11CF11CC801B7010E94842C4DE0E42EF12CEC0EFD1EC701B801FA
:2025A0000E943E2EC70160E048EE53E00E948011C7010E94522E8FEF80935C03CC24DD249E
:2025C0008E010F5F1F4F35E2632E712C6C0E7D1E2FE1822E912C8C0E9D1E93E1A92EB12C3C
:2025E000AC0EBD1E89E1E82EF12CEC0EFD1E08C08091BA03882321F40E942B080E94B70E02
:202600000E94441F8823A1F30E94511F8D3009F476C08F3729F5C114D10491F30894C108FD
:20262000D1082D813E8121503040C501B80140E050E00E94E02DC801B5010E94272EC501B9
:202640000E94522EC701B8010E943E2EC70161E048EE53E00E948011C7010E94522ED0CF9B
:202660008B3109F44FC0682F772767FD7095CB01815690404A9728F0CB01805E90404F9728
:2026800010F4605270406E39710519F46EE870E005C06A39710511F46AE870E0562EC80132
:2026A0000E94B52C2D813E812131310578F0A90140515040C401B8010E94E02DC40161E03C
:2026C00048EE53E00E948011C4010BC0C301B8010E943E2EC30161E048EE53E00E948011A2
:2026E000C3010E94522EF101EC0DFD1D50820894C11CD11C32E5C316D1040CF481CF00E0C2
:2027000010E015C081E08093D2032FC0F101E00FF11F8DEA95E0B70140810E9435248BA937
:202720009CA9E816F90609F486010F5F1F4FE9A8FAA8E00EF11E0C151D0544F38DEA95E061
:20274000B7014FEF0E9435248E01055D1F4FC8016DE572E00E94352DC80160E048EE53E046
:202760000E948011C8010E94522ECE0107960E94522ECE0101960E94522E842D9FA90FB667
:20278000F8949EBF0FBE8DBF2DA93EA90FB6F8943EBF0FBE2DBFE7960FB6F894DEBF0FBE3B
:2027A000CDBFCF91DF911F910F91FF90EF90DF90CF90BF90AF909F908F907F906F905F90B8
:2027C0004F903F902F9008958091D203813071F58091D7038093D203882321F0833009F0B7
:2027E00064C003C00E947911089584E994E00E94E32084E994E060E040E00E94B42084E97F
:2028000094E069ED73E00E94FD2884E994E060E041E00E94B42084E994E06FED73E00E94EA
:20282000FD281092E5031092D8030895823019F08330D9F512C00E9406252091D3033091AC
:20284000D4034091D5035091D603261737074807590718F481E08093D2038091D803882328
:2028600021F18091E503882331F084E994E00E94E3201092E50384E994E060E040E00E948E
:20288000B42084E994E069ED73E00E94FD2884E994E060E041E00E94B42084E994E06FED1E
:2028A00073E00E94FD281092D8030895CF92DF92EF92FF920F931F93DF93CF93CDB7DEB7BF
:2028C00062970FB6F894DEBF0FBECDBF082F80935C0357E0C52ED12CCC0EDD1EC60162E604
:2028E00072E00E944E2D10E00F5F1F4F7E010894E11CF11CC701B8014AE00E94B02DC60187
:20290000B7010E94FE2CBC018E01035F1F4FC8010E943E2EC80160E048EE53E00E9480119B
:20292000C8010E94522EC7010E94522EC6010E94582E0E94E41362960FB6F894DEBF0FBE87
:20294000CDBFCF91DF911F910F91FF90EF90DF90CF9008951F93182F8091D203833039F097
:2029600083E08093D20384E994E00E94E3208091B5048031E8F08091B4048F5F8093B404B1
:202980001092B5048230A0F089ED93E06FED73E00E94272E8FED93E060E071E00E94672D55
:2029A0008091B40481508093B40481E08093E5038091B40426E0829FC001112487529C4FAC
:2029C000612F0E94B52C8091B5048F5F8093B50481E08093D8031F9108958F929F92AF9231
:2029E000BF92CF92DF92FF920F931F93DF93CF93CDB7DEB72C970FB6F894DEBF0FBECDBFD8
:202A0000182F8C3018F00E94EB0BC5C0CE01019660E071E00E94352D10928D041092BF03FC
:202A20008091BA03882331F48091A9049091AA040E940F2982E5189FC00111247EE1A72E49
:202A4000B12CA80EB91E85016FE6C62ED12CC80ED91E46010894811C911C95C08091BA0323
:202A6000882321F40E94E0190E94E4130E94620B80918D04882309F072C08091C903882353
:202A800009F06DC08DEA95E0B8010E942E24F82E8FEFF81609F44CC08CE5F81669F18091D2
:202AA000BA038823C9F48091F403882361F4E091A904F091AA04A081B1812D913C91CF01EE
:202AC0006F2DF901099580915B03882329F08F2D0E94AA140E94E4138091AB04882339F046
:202AE0008F2D61E00E94C40F1092AB0407C08F2D60E00E94C40F02C00F5F1F4F8091BA036F
:202B00008130A9F18091BD03882341F48091BE03882321F48091BF03882349F11092BD030D
:202B20001092BE031092BF038FEF80935C032FC00A151B0561F5F0925C038E01095F1F4F14
:202B4000C80161E772E00E94352DC80160E048EE53E00E948011C8010E94522E18C0809195
:202B6000C903882311F4840102C0015010400E94062560938E0470938F048093900490933F
:202B800091040F5F1F4FC016D1060CF067CFCE0101960E94522E2C960FB6F894DEBF0FBEE0
:202BA000CDBFCF91DF911F910F91FF90DF90CF90BF90AF909F908F900895CF93DF93282F68
:202BC00010928D0480918C04882309F07CC290918B04992309F4CEC28091C903882309F0C5
:202BE000C9C26091F503862F8E508A3008F021C26531A9F482E080938C04892F8150809365
:202C00008B04882361F0E5EFF3E0282F30E02E0F3F1F02C081818193E217F307D9F78091D4
:202C2000F5038631B9F480918B04882319F0815080938B0480918B04882361F0E5EFF3E02E
:202C4000282F30E02E0F3F1F02C081818193E217F307D9F78091F5038731A1F580918B04E0
:202C6000882319F0815080938B0480918B04882349F1C5EFD3E0FE01282F30E02C0F3D1F44
:202C800002C081818193E217F307D9F78091F5038C3010F40E94ED1480918B04882319F0D9
:202CA000815080938B0480918B04882321F40AC08981899304C0282F30E02B503C4FC21747
:202CC000D307B1F78091F5038E3009F047C080918B04882319F0815080938B0490918B0434
:202CE0009923E1F1A5EFB3E0FD01292F30E02A0F3B1F02C081818193E217F307D9F79230C9
:202D000068F15091F503492F4150E5EFF3E0242F30E02E0F3F1F02C081818193E217F30708
:202D2000D9F7952F80E02091F503820F911D9093970380939603842F815080938B0488237D
:202D400031F40CC011968C9111978D9304C0282F30E02B503C4FA217B307A1F78091F503B1
:202D60008331B9F480918B04882319F0815080938B0480918B04882361F0E5EFF3E0282F91
:202D800030E02E0F3F1F02C081818193E217F307D9F78091F503843109F053C080918B0483
:202DA000882319F0815080938B0480918B04882341F1C5EFD3E0FE01282F30E02C0F3D1F0B
:202DC00002C081818193E217F307D9F78091F50361E00E94C40F80918B04882319F0815074
:202DE00080938B0480918B04882321F40AC08981899304C0282F30E02B503C4FC217D307FD
:202E0000B1F780918B048823E1F08091F50360E00E94C40F80918B04882319F081508093F8
:202E20008B0480918B04882361F0E5EFF3E0282F30E02E0F3F1F02C081818193E217F307F3
:202E4000D9F78091F503813109F059C080918B04882319F0815080938B0480918B048823C3
:202E600009F44DC0C5EFD3E0FE01282F30E02C0F3D1F02C081818193E217F307D9F781E0E8
:202E800080938C0481E090E060E00E94FE0B0E9406252091F50330E048EE53E0F901E49F67
:202EA0009001E59F300DF49F300D1124442737FD4095542F260F371F481F591F2093AD04F6
:202EC0003093AE044093AF045093B00481E18093AC0480918B04882319F0815080938B0474
:202EE00080918B04882321F40AC08981899304C0282F30E02B503C4FC217D307B1F78091E5
:202F0000F503823109F054C080918B04882319F0815080938B0480918B04882309F448C0E2
:202F2000C5EFD3E0FE01282F30E02C0F3D1F02C081818193E217F307D9F781E080938C048E
:202F40000E9406252091F50330E048EE53E0F901E49F9001E59F300DF49F300D1124442743
:202F600037FD4095542F260F371F481F591F2093AD043093AE044093AF045093B00482E102
:202F80008093AC0480918B04882319F0815080938B0480918B04882321F40AC08981899357
:202FA00004C0282F30E02B503C4FC217D307B1F78091F5038F30E1F480918B04882319F094
:202FC000815080938B0480918B04882361F0E5EFF3E0282F30E02E0F3F1F02C08181819361
:202FE000E217F307D9F781E08093B9030E945C0A8091F503803109F0BDC080918B0488235B
:2030000019F0815080938B0480918B04882361F0E5EFF3E0282F30E02E0F3F1F02C081812B
:203020008193E217F307D9F71092B9030E94BA08A1C0222301F58091F4038823E1F4A091A2
:20304000A904B091AA04ED91FC9111970190F081E02DCD0109958091F5038D3061F4E0911A
:20306000A904F091AA04A081B1812D913C91CF016AE0F901099580915B03882331F0809198
:20308000F5030E94AA140E94E4138091F50360E00E94C40F80918B04882319F08150809349
:2030A0008B0480918B04882309F464C0E5EFF3E0282F30E02E0F3F1F02C081818193E2179B
:2030C000F307D9F757C0813099F58091AC048131C1F40E9406252091AD043091AE04409135
:2030E000AF045091B004261737074807590748F480E090E060E00E94FE0B1092AC04109273
:203100008C048091AC04823199F40E9406252091AD043091AE044091AF045091B004261726
:2031200037074807590720F41092AC0410928C0490918C049230F1F480918B04882329F04E
:2031400020E030E0682F70E00FC010928C0412C0F901EB50FC4F8081863111F0A90101C001
:2031600090E09A012F5F3F4FAB012617370784F390938C040E942B088091BD03882321F471
:203180008091BE03882379F080918B04882359F010928B0410928C041092BD031092BE038D
:2031A0008FEF80935C03DF91CF9108952F923F924F925F926F927F928F929F92AF92BF9258
:2031C000CF92DF92EF92FF920F931F93DF93CF93CDB7DEB7AE970FB6F894DEBF0FBECDBF3E
:2031E000E82E7CA76BA75EA74DA78E010F5F1F4FC80160E071E00E94352D8FEF80935C03D2
:20320000FF24A3E12A2E312C2C0E3D1E5801F9E14F2E512C4C0E5D1EE7E06E2E712C6C0E41
:203220007D1E7DE0872E912C8C0E9D1E0E94441F882379F48091BA03882309F065C00E9479
:203240002B080E94B70E80E00E94DD150E94FD095BC00E94511F682F80538A3068F5C62E96
:20326000DD24C7FCD0941F2D1F5FB60160537040C3014AE00E94B02DC501B3010E94C82CC5
:20328000C3010E94522EC401B5010E943E2EC40161E048EE53E00E948011C4010E94522E36
:2032A000E11608F45CC0EF2DF0E0EE0FFF1FEA0DFB1DD78EC68E29C06F3719F5FF2021F162
:2032C0001F2D11502D813E8121503040C101B50140E050E00E94E02DC501B1010E94272E0D
:2032E000C1010E94522EC201B5010E943E2EC20161E048EE53E00E948011C2010E94522EDE
:2033000004C06D3061F54DC01F2DF12E8FCF8D919C911197C097AC01249FC001259F900D44
:20332000349F900D1124080F191FC901880F991F43E0220F331F4A95E1F7280F391F3197CC
:2033400012975FEFEF3FF50711F78BA59CA5801791072CF44DA55EA50417150724F00E94A2
:20336000EB0B0FEF1FEFCE0101960E94522EC801AE960FB6F894DEBF0FBECDBFCF91DF919F
:203380001F910F91FF90EF90DF90CF90BF90AF909F908F907F906F905F904F903F902F90BB
:2033A0000895EF2DF0E03197DE015F96CF01880F991FA80FB91F21E030E000E010E0C1CFC9
:2033C0002F923F924F925F926F927F928F929F92AF92BF92CF92DF92EF92FF920F931F935B
:2033E000DF93CF93CDB7DEB7CA58D0400FB6F894DEBF0FBECDBF37E6432E512C4C0E5D1E87
:2034000021E6222E312C2C0E3D1E99E4A92EB12CAC0EBD1E83E4882E912C8C0E9D1E0DE37E
:20342000602E712C6C0E7D1E4BC3822F90E0FC013897EC3CF10508F000C3E955FF4FEE0FEF
:20344000FF1F0590F491E02D099480919B0390919C039C012C5E3F4F8851914009C08091E2
:203460009B0390919C039C012451304080549140855A964008F024C330939C0320939B0380
:20348000D9C120919D0330919E03C9016AE070E00E94C032620F731FCB018759904083598C
:2034A000924008F0C7C170939E0360939D03C2C120919D0330919E03C9016AE070E00E9447
:2034C000C032261B370BC901875990408359924008F0B0C130939E0320939D03ABC18091B2
:2034E000960390919703019605C0809196039091970301970E94FF11E3C28CE291E09093C6
:203500009E0380939D0381E08093BC0331C28091C903882319F01092C903D2C281E080932A
:20352000C9038E010F5F1F4FC8016EE772E068C081E08093B204C4C280E001C081E00E94E8
:203540001504BEC282E0FBCF83E0F9CF84E0F7CF85E0F5CF86E0F3CF87E0F1CF88E0EFCFB3
:2035600089E0EDCF8AE0EBCF8BE0E9CF80E015C081E013C082E011C083E00FC084E00DC0E0
:2035800085E00BC086E009C087E007C088E005C089E003C08AE001C08BE00E94561490C251
:2035A00080918B04882309F48BC2815080938B0487C28091B903882321F01092B9030E9431
:2035C000BA088091B304882339F080E090E061E00E94FE0B1092B3048091C903882311F0EF
:2035E0001092C90310928B0481E080938D048FEF80935C038E01095F1F4FC80164E872E06B
:203600000E94352DC80160E048EE53E00E948011C80110C280E015C081E013C082E011C0CA
:2036200083E00FC084E00DC085E00BC086E009C087E007C088E005C089E003C08AE001C016
:203640008BE00E9452123CC20E94D81080915603909157030196909357038093560330C21A
:203660000E94D8102DC280915603909157030197909357038093560313E1C12ED12CCC0EB1
:20368000DD1EC6016AE872E00E944E2DBDE0EB2EF12CEC0EFD1E6091560370915703C70152
:2036A0004AE00E94802DC601B7010E94FE2CBC018E01075E1F4FC8010E943E2EC80160E047
:2036C00048EE53E00E948011C8010E94522EC7010E94522EC6010E94582EF2C183E0809361
:2036E00099038E01015E1F4FC80163E972E03EC082E0809399038E010B5D1F4FC8016CE9D9
:2037000072E034C085E0809399038E01055D1F4FC80165EA72E02AC08E010F5C1F4FC8016B
:203720006FEA72E00E94352DC80160E048EE53E00E948011C8010E94522E84E060E070E056
:2037400040E157E20E94D618181619060CF0B8C19093570380935603CFC084E08093990332
:203760008E01095C1F4FC8016EEB72E00E94352DC80160E048EE53E00E948011C80158C0E9
:203780008091BB03882321F481E08093BB0302C01092BB030E948B0B93C18091BC0388233F
:2037A00079F01092BC03C30162EC72E00E94352DC30160E048EE53E00E948011C3013AC178
:2037C00081E08093BC03C40169EC72E00E94352DC40160E048EE53E00E948011C4012AC1F5
:2037E00080919803882381F481E080939803C5016FEC72E00E94352DC50160E048EE53E008
:203800000E948011C50114C010929803CE01815B9F4F6EED72E00E94352DCE01815B9F4FBB
:2038200060E048EE53E00E948011CE01815B9F4F0E94522E81E09CC080919A038150823003
:20384000A8F410929A03CE018B5A9F4F6CEE72E00E94352DCE018B5A9F4F60E048EE53E0F0
:203860000E948011CE018B5A9F4FE2CFCE01855A9F4F69EF72E00E94352DCE01855A9F4FDC
:2038800060E048EE53E00E948011CE01855A9F4F0E94522E81E080939A03CCCF8FEF809351
:2038A0005C038091B304882341F080E090E061E00E94FE0B1092B3041FC0C10165E073E0B7
:2038C0000E94352DC10160E048EE53E00E948011C1010E94522E81E090E061E00E94FE0BA5
:2038E00081E08093B304ECC08091C703882341F01092B9030E94BA0881E08093D203E0C08F
:20390000C2016AE073E00E94352DC20160E048EE53E00E948011C2010E94522E81E080934B
:20392000B9030E945C0ACCC0CE0183599F4F65E173E00E94352DCE0183599F4F60E048EEF2
:2039400053E00E948011CE0183599F4F0E94522E83E060E070E048EE53E00E94D61818162C
:2039600019060CF0ADC00E94FF1181E08093D2038093C203A5C081E00E943304CE018D5899
:203980009F4F6FE372E00E94352DCE018D589F4F60E048EE53E00E948011CE018D589F4F71
:2039A00049C082E00E943304CE0187589F4F64E472E00E94352DCE0187589F4F60E048EE77
:2039C00053E00E948011CE0187589F4F33C08091A1038823C1F01092A10381E08093C20362
:2039E000CE0181589F4F60E273E00E94352DCE0181589F4F60E048EE53E00E948011CE0157
:203A000081589F4F17C081E08093A1038093C203CE018B579F4F6EE273E00E94352DCE0103
:203A20008B579F4F60E048EE53E00E948011CE018B579F4F0E94522E43C0822F80528B35D3
:203A400008F03EC08091B204882371F0E0918B04E63940F4EF5FE0938B04F0E0EC50FC4FA3
:203A600084E180831092B20430E0C901815690404A9728F0C901805E90404F9710F4205238
:203A800030402E39310519F42EE830E005C02A39310511F42AE830E0E0918B04E63968F4E6
:203AA0002F3741F0EF5FE0938B04F0E0EC50FC4F208303C0E150E0938B048FEF80935C033F
:203AC0000E94441F882361F080918D04882341F40E94511F282F80919204882389F7A5CCB7
:203AE000C657DF4F0FB6F894DEBF0FBECDBFCF91DF911F910F91FF90EF90DF90CF90BF90E9
:203B0000AF909F908F907F906F905F904F903F902F9008956F927F928F929F92AF92BF921B
:203B2000CF92DF92EF92FF920F931F938091E6039091E703A091E803B091E9030097A105C2
:203B4000B10509F45EC080915A03882309F459C00E9406252091EA033091EB034091EC038B
:203B60005091ED03261737074807590708F049C06091E6037091E7038091E8039091E9037B
:203B80000E944F040E94AA141092E6031092E7031092E8031092E9030E9406250E94883176
:203BA0005B016C01609196037091970388E592E00E94C03280E090E00E9488317B018C0170
:203BC0006091580370E0882777FD8095982F0E948A319B01AC01C801B7010E943E329B0175
:203BE000AC01C601B5010E9487300E945C316093EA037093EB038093EC039093ED0310928B
:203C00005D038091E6039091E703A091E803B091E9030097A105B10509F050C080915A038C
:203C2000882309F44BC00E9406250E9488313B014C016091EA037091EB038091EC03909132
:203C4000ED030E9488315B016C01609196037091970380EB94E00E94C03280E090E00E9446
:203C600088317B018C016091A00370E020915803621B7109882777FD8095982F0E948A313F
:203C80009B01AC01C801B7010E943E329B01AC01C601B5010E9487309B01AC01C401B30167
:203CA0000E943A32181654F480915D03882331F480E20E94AA1481E080935D031F910F9159
:203CC000FF90EF90DF90CF90BF90AF909F908F907F906F9008958091BA03882301F50E9470
:203CE0002B080E94B70E0E94620B0E942B080E94B70E80E00E94DD150E94FD090E94E019A8
:203D00000E940F0B0E94820A0E942B080E94B70E80E00E94DD150E948A1D0E94E41308950A
:203D20004091BA04E091B8048091B704E81771F08E2F8F5F8D3208F080E0E82FF0E0E554B9
:203D4000FB4FE0818093B804EE2321F44093BA0480E00895E03F11F44160E4CFE03E11F49A
:203D60004260E0CF242F30E040FF11C0E23111F44B7F0BC0E93511F4477F07C0E43111F408
:203D80004F7E03C0E13109F44F7D4C7FCBCFE23111F44460C7CFE93511F44860C3CFE4318F
:203DA00011F44061BFCFE13111F44062BBCF41FF3EC0E03721F1E13780F4E93641F1EA3628
:203DC00030F4EA3481F1EA3509F056C02EC0EB3621F1EC3609F050C014C0E43711F1E537A8
:203DE00030F4E13791F0E23709F046C018C0EA3781F0ED3741F0E53709F03EC00CC080E8E8
:203E00003CC081E83AC089E138C08FE736C08CE934C08AE132C08BE030C088E02EC08AE094
:203E20002CC085E12AC08FE228C08DE026C0C9018C709070892B39F0E438F0F4F0E0EC54E7
:203E4000FB4F84911AC044FF07C0E438A8F4F0E0E85CFA4F849111C045FF07C0E43860F4A9
:203E6000F0E0E454FA4F849108C0E43828F4F0E0E05CF94F849101C080E04C7F882309F4DF
:203E800051CF4093BA0408958091B904882311F081E008950E94901E8093B904811181E049
:203EA00008958091B904882319F01092B90407C00E94901E882319F42FEF3FEF04C0282F4E
:203EC000332727FD3095C901089508950F931F93182F062F8093B604862F62E00E94B2258E
:203EE000812F62E00E94B225033011F481E001C080E01092B7041092B80466E87FE142E012
:203F000050E00E9441241F910F910895CF92DF92EF92FF921F938091B6040E944526182FC8
:203F20000E9406259B01AC018091E8049091E904A091EA04B091EB0469017A01C81AD90A67
:203F4000EA0AFB0AD701C6018B3F9105A105B10520F01092ED041092EC042093E804309376
:203F6000E9044093EA045093EB043091ED04232F2150283060F4812F90E002C0880F991F6F
:203F80002A95E2F72091EC04282B2093EC04832F8F5F8093ED048B30B9F49091B7049F5F0C
:203FA0009D3208F090E08091B804981749F0E92FF0E08091EC04E554FB4F80839093B704C8
:203FC0001092ED041092EC041F91FF90EF90DF90CF9008950F931F938C01FC01868160E06E
:203FE0000E94F12581E090E00E946D25F801868161E00E94F12581E090E00E946D25F8010D
:20400000868160E00E94F12584E690E00E946D251F910F910895CF92DF92EF92FF920F9320
:204020001F93CF93DF93D82EC92E282F392FC9018C01C0E0D0E0E62EFF24F801878161E01E
:204040000E94B225B7010C2E02C0759567950A94E2F76170F80187810E94F12521960F5F07
:204060001F4FC830D10549F78D2D9C2D0E94EA1FDF91CF911F910F91FF90EF90DF90CF909A
:204080000895CF92DF92EF92FF920F931F93CF93DF93D82EC92E282F392FC9018C01C0E0C4
:2040A000D0E0E62EFF24F801878161E00E94B225B7010C2E02C0759567950A94E2F761705C
:2040C000F80187810E94F12521960F5F1F4FC430D10549F78D2D9C2D0E94EA1FDF91CF918C
:2040E0001F910F91FF90EF90DF90CF9008951F93CF93DF93EC01162F8C81642F0E94F125E7
:204100008D818F3F19F060E00E94F1258F8584FF05C0CE01612F0E940B200EC0612F70E08C
:2041200084E0759567958A95E1F7CE010E944120CE01612F0E944120DF91CF911F910895CD
:2041400041E00E94772081E090E0089540E00E9477200895FC016089862F8460808B6C604B
:20416000CF010E94A6200895DF93CF93CDB7DEB728970FB6F894DEBF0FBECDBF9C01FE01DB
:204180003196ADE6B3E088E00D9001928150E1F7F9018389481710F0482F4150E42FF0E0A1
:2041A000EE0FFF1FEC0FFD1F8181680F6068C9010E94A62028960FB6F894DEBF0FBECDBF55
:2041C000CF91DF91089561E00E94A62080ED97E00E946D250895CF93DF93EC01423018F0D9
:2041E0008F8588608F874B8B1C8A222329F0413019F48F8584608F8780E593EC0E946D252F
:204200008C8160E00E94F1258E8160E00E94F1258D818F3F19F060E00E94F1256F8564FD60
:204220001DC0CE0163E00E94412084E991E10E946D25CE0163E00E94412084E991E10E94E3
:204240006D25CE0163E00E94412086E990E00E946D25CE0162E00E94412016C06062CE0129
:204260000E94A62084E991E10E946D256F856062CE010E94A62086E990E00E946D256F85CF
:204280006062CE010E94A6206F856062CE010E94A62084E0888BCE010E94AA20CE010E9415
:2042A000E32082E0898BCE0166E00E94A620DF91CF9108956F927F928F92AF92CF92EF9245
:2042C0000F931F93DF93CF93CDB7DEB73C01162F842FF301448325830683E782C086A186A6
:2042E00082869D8593879E8594879F8595879889968761E00E94B225F30185818F3F19F033
:2043000061E00E94B225F301868161E00E94B225112319F0F301178603C080E1F30187873A
:20432000C30160E141E020E00E94EB20CF91DF911F910F91EF90CF90AF908F907F906F9040
:2043400008958F92AF92CF92EF920F931F93CF93DF93DC01362F542F722F102FAE2C8C2C1D
:2043600013961C921E92129789E693E011969C938E9300D000D0EDB7FEB73196CDB7DEB7DB
:204380001982118212821382CD0161E0432F2FEF052FE72EC12E0E945A210F900F900F90F5
:2043A0000F90DF91CF911F910F91EF90CF90AF908F90089520910F0530E080910E05281B29
:2043C0003109C901089540910E0580910F05481718F02FEF3FEF0AC0E42FF0E0E251FB4F56
:2043E0008081282F30E04F5F40930E05C9010895E0910E0580910F05E81718F0EFEFFFEFDE
:2044000006C0F0E0E251FB4F8081E82FF0E0CF0108950895109236051092350588EE93E0F5
:20442000A0E0B0E08093370590933805A0933905B0933A0589E793E0909334058093330540
:204440000895CF92DF92EF92FF920F931F93CF93DF937C016B018A01809132058823A1F0BB
:20446000C0E0D0E00DC0D701ED91FC91D601AC0FBD1F0190F081E02DC7016C9109952196A5
:20448000C017D10780F304C0CB01642F0E948222C801DF91CF911F910F91FF90EF90DF902B
:2044A000CF900895DF93CF930F92CDB7DEB7FC016983809132058823C9F0809131058032E4
:2044C00038F081E090E09383828320E030E015C080913005E82FF0E0E05FFA4F9981908301
:2044E0008F5F809330058093310505C0CE01019661E00E94822221E030E0C9010F90CF91B1
:20450000DF910895482F613210F081E0089580913F05843011F082E0089560938A05A9E66C
:20452000B5E0842F9C01F90102C081918D938E2F841B8617D0F380E008951F920F920FB6D8
:204540000F9211242F933F934F935F936F937F938F939F93AF93BF93EF93FF938091B90043
:2045600090E0887F90708036910509F4F2C081369105CCF58832910509F47BC089329105E2
:20458000B4F48031910509F46FC0813191053CF4009709F447C1089709F04FC165C0883166
:2045A000910509F466C0809709F047C182C08034910509F4A4C08134910544F48033910571
:2045C00009F482C0C89709F038C189C08035910509F489C08835910509F496C08834910579
:2045E00009F02BC1AEC08839910509F413C189399105ECF48837910509F4ABC089379105F5
:204600004CF48836910509F4A4C08037910509F014C19FC08838910509F4FCC080399105CD
:2046200009F49DC08038910509F007C198C0803B910509F4C6C0813B91054CF4803A910503
:2046400009F49FC0883A910509F0F7C0BAC0803C910509F4E3C0883C910509F4DFC0883BD1
:20466000910509F0EAC0C2C0809140058093BB00CFC09091670580916805981768F4909195
:204680006705E92FF0E0E95BFA4F80818093BB009F5F90936705BCC080914105882309F462
:2046A0004BC085ED8093BC008091BC0084FDFCCFC2C080E28093AC0585ED8093BC0080919B
:2046C000BC0084FDFCCFB7C080E38093AC0585ED8093BC008091BC0084FDFCCFACC088E303
:2046E0008093AC059BC0809167059091BB00E82FF0E0E95BFA4F90838F5F8093670590912D
:2047000067058091680582C0809167059091BB00E82FF0E0E95BFA4F90838F5F8093670520
:2047200080914105882341F085ED8093BC008091BC0084FDFCCF7FC081E08093420584EA84
:204740006EC085ED8093BC008091BC0084FDFCCF72C083E080933F051092AB0559C0809169
:20476000AB05803208F056C08091AB059091BB00E82FF0E0E557FA4F90838F5F8093AB05FC
:2047800047C08091AB05803230F4E091AB05F0E0E557FA4F108285ED8093BC008091BC0065
:2047A00084FDFCCF10923F056091AB05E0914505F09146058BE895E070E009951092AB0577
:2047C0002DC084E080933F051092890510928A05E0914305F0914405099580918A05882364
:2047E00029F481E080938A051092690590918905E92FF0E0E759FA4F80818093BB009F5F9C
:20480000909389059091890580918A05981710F485EC01C085E88093BC000FC085EC809324
:20482000BC0009C01092AC0585ED8093BC008091BC0084FDFCCF10923F05FF91EF91BF9100
:20484000AF919F918F917F916F915F914F913F912F910F900FBE0F901F901895F999FECF92
:2048600072BD61BDF89A80B50895F999FECF1FBA72BD61BD40BD0FB6F894FA9AF99A0FBEC0
:204880000895823000F5E82FF0E0EE0FFF1FE255FA4F71836083882319F08130A1F408C0B9
:2048A000809169008C7F842B80936900E89A089580916900440F551F440F551F837F842B70
:2048C00080936900E99A08951F920F920FB60F9211242F933F934F935F936F937F938F93B1
:2048E0009F93AF93BF93EF93FF938091AE059091AF05892B29F0E091AE05F091AF05099581
:20490000FF91EF91BF91AF919F918F917F916F915F914F913F912F910F900FBE0F901F907D
:2049200018951F920F920FB60F9211242F933F934F935F936F937F938F939F93AF93BF9379
:20494000EF93FF938091B0059091B105892B29F0E091B005F091B1050995FF91EF91BF917E
:20496000AF919F918F917F916F915F914F913F912F910F900FBE0F901F9018951F920F927E
:204980000FB60F9211242F933F938F939F93AF93BF938091B6059091B705A091B805B09128
:2049A000B9053091BA050196A11DB11D232F2D5F2D3720F02D570196A11DB11D2093BA052B
:2049C0008093B6059093B705A093B805B093B9058091B2059091B305A091B405B091B505B3
:2049E0000196A11DB11D8093B2059093B305A093B405B093B505BF91AF919F918F913F9156
:204A00002F910F900FBE0F901F9018958FB7F8942091B6053091B7054091B8055091B90587
:204A20008FBFB901CA0108959B01AC017FB7F8948091B2059091B305A091B405B091B50575
:204A400066B5A89B05C06F3F19F00196A11DB11D7FBFBA2FA92F982F8827860F911DA11DE3
:204A6000B11D62E0880F991FAA1FBB1F6A95D1F7BC012DC0FFB7F8948091B2059091B305E0
:204A8000A091B405B091B505E6B5A89B05C0EF3F19F00196A11DB11DFFBFBA2FA92F982FEE
:204AA00088278E0F911DA11DB11DE2E0880F991FAA1FBB1FEA95D1F7861B970B885E934079
:204AC000C8F2215030404040504068517C4F211531054105510571F60895019739F0880F43
:204AE000991F880F991F02970197F1F70895789484B5826084BD84B5816084BD85B582601A
:204B000085BD85B5816085BDEEE6F0E0808181608083E1E8F0E0108280818260808380815B
:204B200081608083E0E8F0E0808181608083E1EBF0E0808184608083E0EBF0E08081816013
:204B40008083EAE7F0E0808184608083808182608083808181608083808180688083109270
:204B6000C1000895CF93DF93482F50E0CA018A50994FFC0134914E51594FFA01849188230B
:204B800069F190E0880F991FFC01EC53F94FA591B491FC01E253F94FC591D491662351F4FA
:204BA0002FB7F8948C91932F909589238C93888189230BC0623061F42FB7F8948C91932FFC
:204BC000909589238C938881832B88832FBF06C09FB7F8948C91832B8C939FBFDF91CF9175
:204BE0000895482F50E0CA01865F984FFC012491CA018A50994FFC0194914E51594FFA0137
:204C00003491332309F440C0222351F1233071F0243028F42130A1F0223011F514C026306D
:204C2000B1F02730C1F02430D9F404C0809180008F7703C0809180008F7D8093800010C08C
:204C400084B58F7702C084B58F7D84BD09C08091B0008F7703C08091B0008F7D8093B000EA
:204C6000E32FF0E0EE0FFF1FE253F94FA591B4912FB7F894662321F48C919095892302C07F
:204C80008C91892B8C932FBF0895682F70E0CB01865F984FFC012491CB018A50994FFC01DD
:204CA00044916E51794FFB019491992319F420E030E03CC0222351F1233071F0243028F4F7
:204CC0002130A1F0223011F514C02630B1F02730C1F02430D9F404C0809180008F7703C088
:204CE000809180008F7D8093800010C084B58F7702C084B58F7D84BD09C08091B0008F779D
:204D000003C08091B0008F7D8093B000892F90E0880F991F8852994FFC01A591B4918C9172
:204D200020E030E0842311F021E030E0C901089508951F920F920FB60F9211242F933F9325
:204D40004F938F939F93EF93FF938091C00082FD1DC04091C6002091FB053091FC052F5F44
:204D60003F4F2F7330708091FD059091FE052817390771F0E091FB05F091FC05E554FA4FD7
:204D800040833093FC052093FB0502C08091C600FF91EF919F918F914F913F912F910F90D1
:204DA0000FBE0F901F901895E0914F06F0915006E05CFF4F8191919120813181805C9F4FB3
:204DC000821B930B60E470E00E94D432892B11F00E94982608951F920F920FB60F921124BD
:204DE0002F933F938F939F93EF93FF9320913F06309140068091410690914206281739077A
:204E000031F48091C1008F7D8093C10014C0E0914106F0914206E150FA4F208180914106F3
:204E20009091420601968F73907090934206809341062093C600FF91EF919F918F913F9102
:204E40002F910F900FBE0F901F901895AF92BF92DF92EF92FF920F931F93CF93DF93EC0101
:204E60007A018B01DD24403081EE580780E0680780E0780711F0DD24D39491E0A92EB12CB0
:204E8000EC89FD89DD2069F0C50108A002C0880F991F0A94E2F7808360E079E08DE390E04F
:204EA00005C0108260E874E88EE190E0A80197010E94E73221503040404050405695479564
:204EC0003795279580E12030380720F0DD2011F0DD24D6CFE889F9893083EA89FB89208366
:204EE00019A2EE89FF89408121E030E0C9010C8C02C0880F991F0A94E2F7482B4083EE898F
:204F0000FF894081C9010D8C02C0880F991F0A94E2F7482B4083EE89FF894081C9010E8C03
:204F200002C0880F991F0A94E2F7482B4083EE89FF8980810F8C02C0220F331F0A94E2F75C
:204F4000209528232083DF91CF911F910F91FF90EF90DF90BF90AF900895DC011C96ED91D9
:204F6000FC911D97E05CFF4F8191919120813181805C9F4F821B930B60E470E00E94D4329E
:204F80000895DC011C96ED91FC911D97E05CFF4F20813181E054F040DF01AE5BBF4F8D91D0
:204FA0009C9111972817390719F42FEF3FEF07C08D919C91E80FF91F8081282F30E0C901F1
:204FC0000895DC011C96ED91FC911D97E05CFF4F20813181E054F040DF01AE5BBF4F8D9190
:204FE0009C9111972817390719F42FEF3FEF10C08D919C911197E80FF91F20818D919C9146
:20500000119701968F73907011969C938E9330E0C9010895DC0191968C919197882339F0C4
:205020005496ED91FC915597808186FFF9CF91961C920895CF93DF93EC01EE85FF85E05CDB
:20504000FF4F20813181E054F0402F5F3F4F2F733070DF01AE5BBF4F8D919C9111972817C4
:205060003907D1F3E05CFF4F80819181E054F040E80FF91F6083EE85FF85E05CFF4F318304
:205080002083EE89FF89208181E090E00F8C02C0880F991F0A94E2F7282B208381E089A356
:2050A000EC89FD8980818064808381E090E0DF91CF910895109246061092450688EE93E00B
:2050C000A0E0B0E08093470690934806A0934906B0934A0689E893E090934406809343062D
:2050E0008BEB95E09093500680934F068FEF95E0909352068093510685EC90E090935406AE
:205100008093530684EC90E0909356068093550680EC90E0909358068093570681EC90E0AC
:2051200090935A068093590682EC90E090935C0680935B0686EC90E090935E0680935D06C4
:2051400084E080935F0683E08093600687E08093610685E08093620681E08093630608955C
:20516000CF92DF92EF92FF920F931F93CF93DF937C016B018A01C0E0D0E00FC0D6016D91BB
:205180006D01D701ED91FC910190F081E02DC7010995C80FD91F015010400115110571F745
:2051A000CE01DF91CF911F910F91FF90EF90DF90CF900895EF92FF920F931F93CF93DF934D
:2051C0007C018B01C0E0D0E0F8010F5F1F4F6491662359F0D701ED91FC910190F081E02DE8
:2051E000C7010995C80FD91FEFCFCE01DF91CF911F910F91FF90EF900895CF93DF93FB0152
:20520000EC01A881B98160817181448155811296ED91FC9113970995DF91CF910895EF92E7
:20522000FF920F931F938C01DC01ED91FC910190F081E02D6DE009957C01D801ED91FC91B9
:205240000190F081E02DC8016AE009959C012E0D3F1DC9011F910F91FF90EF900895EF9214
:20526000FF920F931F937C010E94DA288C01C7010E940F299C01200F311FC9011F910F91C3
:20528000FF90EF900895CF93DF93EC016115710519F420E030E00FC0DB010D900020E9F751
:2052A0001197A61BB70BE881F9810280F381E02DAD0109959C01C901DF91CF9108950E941B
:2052C00043290895813041F0813018F08230D1F409C010926E00089580916F008D7F80939E
:2052E0006F000895809170008D7F8093700081E08093B0008091B100887F84608093B100FD
:205300001092B30008951F93182F80915E03811711F09FEF06C0EEE1F7E094918FEF8093E7
:205320005E03892F0E946229812F60E00E94F1251F9108951F920F920FB60F9211242F9383
:205340003F934F935F936F937F938F939F93AF93BF93EF93FF938091730690917406A09141
:205360007506B09176060097A105B10551F1E0917706F0917806808190917906892780837F
:205380008091730690917406A0917506B0917606181619061A061B06C4F48091730690918E
:2053A0007406A0917506B09176060197A109B1098093730690937406A0937506B093760678
:2053C00004C080915E030E948329FF91EF91BF91AF919F918F917F916F915F914F913F91A9
:2053E0002F910F900FBE0F901F9018952F923F925F926F927F928F929F92AF92BF92CF92AC
:20540000DF92EF92FF920F931F93DF93CF9300D000D0CDB7DEB7A82F1B0129833A834B83FE
:205420005C8380915E038A1721F4EEE1F7E0549082C08F3F09F0DAC1A0935E03EEE1F7E0FD
:2054400054902FEF521609F4D1C181E0581639F192E0591609F449C0552009F06CC014BC09
:2054600015BC84B5826084BD85B5816085BD2A2F30E0F901EE51F94FE491F0E0EE0FFF1F58
:20548000E253F94F8591949190936A06809369062A50394FF901849180936B064EC01092FA
:2054A00080001092810080918100886080938100809181008160809381002A2F30E0F901D1
:2054C000EE51F94FE491F0E0EE0FFF1FE253F94F8591949190937106809370062A50394F08
:2054E000F90184918093720628C01092B0001092B1008091B00082608093B0008091B1005D
:2055000081608093B1002A2F30E0F901EE51F94FE491F0E0EE0FFF1FE253F94F85919491E4
:2055200090937806809377062A50394FF90184918093790602C057FC59C18A2F61E00E94CC
:20554000B225552021F0F2E05F1609F0BEC031018824992460E072E18AE790E0A4019301E8
:205560000E94093359016A01860175010894E108F108010911092FEFE216F10401051105C2
:2055800009F008F499C060E472E48FE090E0A40193010E94093379018A010894E108F108AA
:2055A0000109110982E05816C1F49FEFE916F1040105110509F008F484C060E970ED83E062
:2055C00090E0A40193010E94093379018A010894E108F1080109110983E0AFEFEA16F104A7
:2055E0000105110509F008F468C068E478EE81E090E0A40193010E94093379018A01089437
:20560000E108F10801091109552011F483E01DC0B2E05B1611F084E018C0EFEFEE16F104B3
:205620000105110509F008F4DFC064E274EF80E090E0A40193010E94093379018A01089489
:20564000E108F1080109110985E0FFEFEF16F1040105110591F188F162E17AE780E090E06C
:20566000A40193010E94093379018A010894E108F10801091109552011F086E001C084E06B
:205680002FEFE216F10401051105B9F0B0F0C601B50120E034E040E050E00E940933790161
:2056A0008A010894E108F10801091109552011F087E008C085E003C081E0552019F485BDCB
:2056C0003AC082E08093B10036C05101CC24DD2460E072E18AE790E0A60195010E940933E2
:2056E00079018A010894E108F1080109110980E0E81680E0F80681E0080780E0180710F454
:2057000091E010C068E478EE81E090E0A60195010E94093379018A010894E108F10801091D
:20572000110993E0A1E05A1631F480918100887F982B9093810089819A81AB81BC810097A1
:20574000A105B10529F48FEF9FEFAFEFBFEF13C0220C331CB10180E090E029813A814B8175
:205760005C810E94A13228EE33E040E050E00E94E732C901DA01E1E05E16A1F0F2E05F16F1
:2057800019F1552099F5E7BC8093650690936606A0936706B093680680916E008260809387
:2057A0006E0024C0F0928900E092880080936C0690936D06A0936E06B0936F0680916F0098
:2057C000826080936F0012C0E092B3008093730690937406A0937506B09376068091700057
:2057E00082608093700002C084E06CCF0F900F900F900F90CF91DF911F910F91FF90EF9039
:20580000DF90CF90BF90AF909F908F907F906F905F903F902F900895FC019B018481958102
:205820006817790728F4608171816115710529F410927A066AE776E002C0620F731FCB0117
:2058400008950F931F93CF93DF93EC018B016F5F7F4F888199810E94A52F009711F480E0D9
:2058600005C0998388831B830A8381E0DF91CF911F910F910895CF93DF93EC01888199810F
:20588000892B29F08A819B818617970760F4CE010E94212C882341F08C819D81892B19F4FF
:2058A000E881F981108281E0DF91CF910895EF92FF920F931F93CF93DF93EC017B016C8115
:2058C0007D81E114F104C1F04115510599F08A01060F171FB8010E943B2C882369F0888155
:2058E00099812C813D81820F931FB7010E94C7031D830C8381E001C080E0DF91CF911F918B
:205900000F91FF90EF900895EF92FF920F931F93DF93CF93CDB7DEB728970FB6F894DEBF3C
:205920000FBECDBF7C01CB018E010F5F1F4FB8014AE050E00E94CE03F80101900020E9F74A
:205940003197E01BF10BC701B801AF010E94572C28960FB6F894DEBF0FBECDBFCF91DF915D
:205960001F910F91FF90EF900895DF93CF9300D0CDB7DEB769831A82BE016F5F7F4F41E06B
:2059800050E00E94572C0F900F90CF91DF910895FB0160817181448155810E94572C0895DB
:2059A000CF93DF93EC0188819981009711F00E940D2F198218821D821C821B821A82DF9172
:2059C000CF9108950F931F93182F092F6115710561F0DB010D900020E9F71197A61BB70B16
:2059E000AD010E94572C882321F4812F902F0E94D02C812F902F1F910F9108950F931F9357
:205A0000182F092FFB0160817181448155810E94572C882321F4812F902F0E94D02C812FFB
:205A2000902F1F910F910895EF92FF920F931F93CF93DF93EC017B018A01BA010E943B2CC8
:205A4000882321F4CE010E94D02C07C01D830C8388819981B7010E94C703CE01DF91CF913D
:205A60001F910F91FF90EF900895CF93DF93EC01198218821B821A821D821C8261157105D3
:205A800051F0DB010D900020E9F71197A61BB70BAD010E94142DDF91CF910895CF93DF934F
:205AA000EC01198218821B821A821D821C826115710551F0DB010D900020E9F71197A61B3F
:205AC000B70BAD010E94142DDF91CF9108950F931F93182F092F6115710559F0DB010D9085
:205AE0000020E9F71197A61BB70BAD010E94142D02C00E94D02C812F902F1F910F9108952E
:205B0000EF92FF920F931F93DF93CF93CDB7DEB761970FB6F894DEBF0FBECDBF8C01CB019A
:205B2000F8011182108213821282158214827E010894E11CF11CB70150E00E94EF03C80187
:205B4000B7010E94672D61960FB6F894DEBF0FBECDBFCF91DF911F910F91FF90EF9008954E
:205B6000EF92FF920F931F93DF93CF93CDB7DEB762970FB6F894DEBF0FBECDBF8C01CB0139
:205B8000F8011182108213821282158214827E010894E11CF11CB70150E00E94CE03C80148
:205BA000B7010E94672D62960FB6F894DEBF0FBECDBFCF91DF911F910F91FF90EF900895ED
:205BC000BF92CF92DF92EF92FF920F931F93CF93DF93082FB92E6B017A01E9012417350702
:205BE00010F4EA017901802F9B2D67E473E00E94352DD60114968D919C9115978E159F0564
:205C0000D0F08C179D0708F4EC01D601ED91FC911197EC0FFD1F108110826D917C916E0D4A
:205C20007F1D802F9B2D0E94672DD601ED91FC91EC0FFD1F1083802F9B2DDF91CF911F9198
:205C40000F91FF90EF90DF90CF90BF900895CF93DF93EC01FB018617970761F060817181C0
:205C60006115710529F0448155810E94142D02C00E94D02CCE01DF91CF910895FC01118275
:205C8000108213821282158214820E94272E0895FC011182108213821282158214820E946E
:205CA000272E0895FC01808191810E940D2F0895FC01808191810E940D2F08950895CF93DD
:205CC000DF930E9477250E945E2E0E94EE11C4EDD6E20E946B1E2097E1F30E94D426F9CFC2
:205CE0000F931F93CF93DF93BC018230910510F462E070E0E0917D06F0917E0640E050E098
:205D0000A0E0B0E024C08081918186179707D0F08617970771F482819381109729F0139661
:205D20009C938E9312972CC090937E0680937D0627C04115510519F08417950718F48D01D4
:205D4000AC01EF01DF01828193819C01F9013097D1F641155105F9F0CA01861B970B843033
:205D6000910580F48A819B810115110521F0F8019383828304C090937E0680937D06FE01A1
:205D8000329645C0FE01E80FF91F619371930297998388833CC080917B0690917C06892B8B
:205DA00041F4809161039091620390937C0680937B0640916303509164034115510541F41A
:205DC0004DB75EB780915F0390916003481B590B20917B0630917C0624173507B0F4CA0191
:205DE000821B930B8617970780F0AB014E5F5F4F8417950750F0420F531F50937C06409344
:205E00007B06F9016193719302C0E0E0F0E0CF01DF91CF911F910F910895CF93DF939C01BF
:205E2000009709F48FC0EC0122971B821A8260917D0670917E066115710581F48881998123
:205E4000820F931F20917B0630917C062817390739F5D0937C06C0937B0674C0DB0140E0F4
:205E600050E0AC17BD0708F1BB83AA83FE0121913191E20FF31FAE17BF0779F48D919C914E
:205E80001197280F391F2E5F3F4F3983288312968D919C9113979B838A834115510571F470
:205EA000D0937E06C0937D064DC012968D919C911397AD01009711F0DC01D3CFDA01139632
:205EC000DC93CE931297FA0121913191E20FF31FCE17DF0769F488819981280F391F2E5F70
:205EE0003F4FFA01318320838A819B8193838283E0E0F0E0DB0112968D919C9113970097E0
:205F000019F0BC01FD01F6CFAB014E5F5F4FDB018D919C91840F951F20917B0630917C060E
:205F20002817390779F4309729F410927E0610927D0602C0138212824250504050937C06D4
:205F400040937B06DF91CF9108956F927F928F929F92AF92BF92CF92DF92EF92FF920F9304
:205F60001F93CF93DF938C01009729F4CB010E94702E8C01BBC08EEFE82E8FEFF82EE00E21
:205F8000F11E4801860E971E8E149F0408F4ACC0D7014D915C91119746175707B8F0453090
:205FA000510508F4A3C0CA0104978617970708F49DC042505040461B570BF40141935193A0
:205FC0006D937C93CF010E940D2F90C05B01A41AB50A3801640E751EA0917D06B0917E0624
:205FE000E0E0F0E0CC24DD2447C0A615B705A9F5CD91DC911197CE0102968A159B0568F192
:20600000CE018A199B09029612962C91129713963C91059758F0F40122833383CA19DB0953
:20602000D183C083D7016D937C9309C04E5F5F4F4C0F5D1FF70151834083C901FC01C114BC
:20604000D10431F0D6011396FC93EE9312974EC0F0937E06E0937D0649C08D919C9111970A
:20606000E817F90708F4FC016D0112968C91129713969C919C01D901109709F0B6CF8091C9
:206080007B0690917C0686159705E9F4E617F707D0F420916303309164032115310541F429
:2060A0002DB73EB780915F0390916003281B390B82169306C8F490927C0680927B06F7016D
:2060C0007183608313C0CB010E94702EEC01009759F0D7014D915C91B8010E94BE03C801B5
:2060E0000E940D2F8E0102C000E010E0C801DF91CF911F910F91FF90EF90DF90CF90BF908D
:20610000AF909F908F907F906F9008955058BB27AA270ED075C166D130F06BD120F031F410
:206120009F3F11F41EF45BC10EF4E095E7FB51C1E92F77D180F3BA17620773078407950735
:2061400018F071F49EF58FC10EF4E0950B2EBA2FA02D0B01B90190010C01CA01A001112484
:20616000FF27591B99F0593F50F4503E68F11A16F040A22F232F342F4427585FF3CF469594
:2061800037952795A795F0405395C9F77EF41F16BA0B620B730B840BBAF09150A1F0FF0F53
:2061A000BB1F661F771F881FC2F70EC0BA0F621F731F841F48F4879577956795B795F79505
:2061C0009E3F08F0B3CF9395880F08F09927EE0F979587950895D9D008F481E008950CD090
:2061E0000FC107D140F0FED030F021F45F3F19F0F0C0511139C1F3C014D198F39923C9F376
:206200005523B1F3951B550BBB27AA2762177307840738F09F5F5F4F220F331F441FAA1F9E
:20622000A9F333D00E2E3AF0E0E830D091505040E695001CCAF729D0FE2F27D0660F771FA0
:20624000881FBB1F261737074807AB07B0E809F0BB0B802DBF01FF2793585F4F2AF09E3FC7
:20626000510568F0B6C000C15F3FECF3983EDCF3869577956795B795F7959F5FC9F7880FC7
:20628000911D9695879597F90895E1E0660F771F881FBB1F621773078407BA0720F0621BC3
:2062A000730B840BBA0BEE1F88F7E095089504D06894B111D9C00895BCD088F09F5790F02C
:2062C000B92F9927B751A0F0D1F0660F771F881F991F1AF0BA95C9F712C0B13081F0C3D083
:2062E000B1E00895C0C0672F782F8827B85F39F0B93FCCF3869577956795B395D9F73EF4A0
:2063000090958095709561957F4F8F4F9F4F0895E89409C097FB3EF49095809570956195D3
:206320007F4F8F4F9F4F9923A9F0F92F96E9BB279395F695879577956795B795F111F8CFF9
:20634000FAF4BB0F11F460FF1BC06F5F7F4F8F4F9F4F16C0882311F096E911C0772321F061
:206360009EE8872F762F05C0662371F096E8862F70E060E02AF09A95660F771F881FDAF7FE
:20638000880F9695879597F90895990F0008550FAA0BE0E8FEEF16161706E807F907C0F08C
:2063A00012161306E407F50798F0621B730B840B950B39F40A2661F0232B242B252B21F453
:2063C00008950A2609F4A140A6958FEF811D811D089597F99F6780E870E060E008959FEFC7
:2063E00080EC089500240A941616170618060906089500240A9412161306140605060895FA
:20640000092E0394000C11F4882352F0BB0F40F4BF2B11F460FF04C06F5F7F4F8F4F9F4F38
:20642000089557FD9058440F551F59F05F3F71F04795880F97FB991F61F09F3F79F0879503
:206440000895121613061406551FF2CF4695F1DF08C0161617061806991FF1CF869571052C
:20646000610508940895E894BB2766277727CB0197F908958ADF08F48FEF08950BD0C0CF11
:20648000B1DF28F0B6DF18F0952309F0A2CFA7CF1124EACFC6DFA0F3959FD1F3950F50E02D
:2064A000551F629FF001729FBB27F00DB11D639FAA27F00DB11DAA1F649F6627B00DA11D46
:2064C000661F829F2227B00DA11D621F739FB00DA11D621F839FA00D611D221F749F3327C8
:2064E000A00D611D231F849F600D211D822F762F6A2F11249F5750408AF0E1F088234AF087
:20650000EE0FFF1FBB1F661F771F881F91505040A9F79E3F510570F05CCFA6CF5F3FECF303
:20652000983EDCF3869577956795B795F795E7959F5FC1F7FE2B880F911D9695879597F944
:206540000895629FD001739FF001829FE00DF11D649FE00DF11D929FF00D839FF00D749F4F
:20656000F00D659FF00D9927729FB00DE11DF91F639FB00DE11DF91FBD01CF011124089544
:20658000AA1BBB1B51E107C0AA1FBB1FA617B70710F0A61BB70B881F991F5A95A9F78095C3
:2065A0009095BC01CD01089597FB092E07260AD077FD04D0E5DF06D000201AF470956195B3
:2065C0007F4F0895F6F7909581959F4F0895A1E21A2EAA1BBB1BFD010DC0AA1FBB1FEE1FBC
:2065E000FF1FA217B307E407F50720F0A21BB30BE40BF50B661F771F881F991F1A9469F721
:2066000060957095809590959B01AC01BD01CF01089597FB092E05260ED057FD04D0D7DF22
:206620000AD0001C38F450954095309521953F4F4F4F5F4F0895F6F790958095709561956A
:206640007F4F8F4F9F4F0895EE0FFF1F0590F491E02D099417E0C6E2D7E004C0FE010E9469
:2066600026332296C832D107C9F7F894FFCF002E2D002D2E2E2E002D2E2D2E002D2E2E00CC
:206680002E002E2E2D2E002D2D2E002E2E2E2E002E2E002E2D2D2D002D2E2D002E2D2E2E85
:2066A000002D2D002D2E002D2D2D002E2D2D2E002D2D2E2D002E2D2E002E2E2E002D002EC5
:2066C0002E2D002E2E2E2D002E2D2D002D2E2E2D002D2E2D2D002D2D2E2E002D2D2D2D2D1E
:2066E000002E2D2D2D2D002E2E2D2D2D002E2E2E2D2D002E2E2E2E2D002E2E2E2E2E002DF9
:206700002E2E2E2E002D2D2E2E2E002D2D2D2E2E002D2D2D2D2E002D2E2E2E2D002D2E2EAB
:206720002D2E002D2E2E2E2D2E2D002E2D2E2D2E2D002D2D2E2E2D2D002E2D2D2D2D2E008E
:206740002D2E2D2E2D2D002D2E2D2D2E002D2E2D2D2E2D002E2D2E2E2E002D2D2D2E2E2E40
:20676000002D2E2D2E2D2E002E2D2E2D2E002D2E2E2E2E2D002E2E2D2D2E2D002E2D2E2E4A
:206780002D2E002E2E2E2D2E2E2D002E2D2D2E2D2E002E2E2E2D2E2D002E2E2D2D2E2E0029
:2067A00020004B334E47204B6579657200545820310054582032002077706D0050726F677F
:2067C00072616D204D656D6F727900446F6E6500526570656174204D656D6F727920004DF3
:2067E000656D6F727920656D7074790050617573650041626F72740053657269616C3A206E
:206800000049616D62696320410049616D626963204200556C74696D6174696300456E7458
:2068200065722053657269616C202300427567005458204F6666005458204F6E005061641B
:20684000646C65205265766572736500506164646C65204E6F726D616C0053696465746FCC
:206860006E65204F66660053696465746F6E65204F6E0054756E650050545420496E766FA2
:206880006B650057504D2041646A757374004175746F7370616365204F6666004175746F30
:2068A0007370616365204F6E0050676D204D656D6F72792000000B0A000A000A000A000AD5
:2068C000000A0001010003010101FF01FF80007F06000000000000A020B0280000400014B6
:2068E0000054000000000052222122DA21E321F8210922000000001A28B028AD27E127C193
:20690000270A2800FFFFFFFFFFFFFFFFFFFFFFFFFFFFFFFFFFFFFFFFFFFFFFFFFFFFFFFF3A
:20692000FFFFFFFFFFFFFFFFFFFFFFFFFFFFFFFFFFFFFFFFFFFFFFFFFFFFFFFFFFFFFFFF77
:20694000FFFFFFFFFFFFFFFFFFFFFFFFFFFFFFFFFFFFFFFFFFFFFFFFFFFFFFFFFFFFFFFF57
:20696000FFFFFFFFFFFFFFFFFFFFFFFFFFFFFFFFFFFFFFFFFFFFFFFFFFFFFFFFFFFFFFFF37
:20698000F92F96E9BB279395F695879577956795B795F111F8CFFAF4BB0F11F460FF1BC08B
:2069A0006F5F7F4F8F4F9F4F16C0882311F096E911C0772321F09EE8872F762F05C06623C3
:2069C00071F096E8862F70E060E02AF09A95660F771F881FDAF7880F9695879597F90895BC
:2069E000990F0008550FAA0BE0E8FEEF16161706E807F907C0F012161306E407F50798F081
:206A0000621B730B840B950B39F40A2661F0232B242B252B21F408950A2609F4A140A695B6
:206A20008FEF811D811D089597F99F6780E870E060E008959FEF80EC089500240A9416164F
:206A4000170618060906089500240A9412161306140605060895092E0394000C11F4882300
:206A600052F0BB0F40F4BF2B11F460FF04C06F5F7F4F8F4F9F4F089557FD9058440F551FBC
:206A800059F05F3F71F04795880F97FB991F61F09F3F79F087950895121613061406551FD1
:206AA000F2CF4695F1DF08C0161617061806991FF1CF86957105610508940895E894BB2735
:206AC00066277727CB0197F908958ADF08F48FEF08950BD0C0CFB1DF28F0B6DF18F09523AB
:206AE00009F0A2CFA7CF1124EACFC6DFA0F3959FD1F3950F50E0551F629FF001729FBB276B
:206B0000F00DB11D639FAA27F00DB11DAA1F649F6627B00DA11D661F829F2227B00DA11DCE
:206B2000621F739FB00DA11D621F839FA00D611D221F749F3327A00D611D231F849F600DCE
:206B4000211D822F762F6A2F11249F5750408AF0E1F088234AF0EE0FFF1FBB1F661F771F0D
:206B6000881F91505040A9F79E3F510570F05CCFA6CF5F3FECF3983EDCF3869577956795E5
:206B8000B795F795E7959F5FC1F7FE2B880F911D9695879597F90895629FD001739FF00134
:206BA000829FE00DF11D649FE00DF11D929FF00D839FF00D749FF00D659FF00D9927729F8C
:206BC000B00DE11DF91F639FB00DE11DF91FBD01CF0111240895AA1BBB1B51E107C0AA1F50
:206BE000BB1FA617B70710F0A61BB70B881F991F5A95A9F780959095BC01CD01089597FBDB
:206C0000092E07260AD077FD04D0E5DF06D000201AF4709561957F4F0895F6F79095819598
:206C20009F4F0895A1E21A2EAA1BBB1BFD010DC0AA1FBB1FEE1FFF1FA217B307E407F50770
:206C400020F0A21BB30BE40BF50B661F771F881F991F1A9469F760957095809590959B0162
:206C6000AC01BD01CF01089597FB092E05260ED057FD04D0D7DF0AD0001C38F450954095B0
:206C8000309521953F4F4F4F5F4F0895F6F790958095709561957F4F8F4F9F4F0895EE0FAC
:206CA000FF1F0590F491E02D099417E0C6E2D7E004C0FE010E9451362296C832D107C9F766
:206CC000F894FFCF002E2D002D2E2E2E002D2E2D2E002D2E2E002E002E2E2D2E002D2D2E9C
:206CE000002E2E2E2E002E2E002E2D2D2D002D2E2D002E2D2E2E002D2D002D2E002D2D2D50
:206D0000002E2D2D2E002D2D2E2D002E2D2E002E2E2E002D002E2E2D002E2E2E2D002E2D2D
:206D20002D002D2E2E2D002D2E2D2D002D2D2E2E002D2D2D2D2D002E2D2D2D2D002E2E2DB9
:206D40002D2D002E2E2E2D2D002E2E2E2E2D002E2E2E2E2E002D2E2E2E2E002D2D2E2E2E61
:206D6000002D2D2D2E2E002D2D2D2D2E002D2E2E2E2D002D2E2E2D2E002D2E2E2E2D2E2D47
:206D8000002E2D2E2D2E2D002D2D2E2E2D2D002E2D2D2D2D2E002D2E2D2E2D2D002D2E2D2A
:206DA0002D2E002D2E2D2D2E2D002E2D2E2E2E002D2D2D2E2E2E002D2E2D2E2D2E002E2D06
:206DC0002E2D2E002D2E2E2E2E2D002E2E2D2D2E2D002E2D2E2E2D2E002E2E2E2D2E2E2DB5
:206DE000002E2D2D2E2D2E002E2E2E2D2E2D002E2E2D2D2E2E0020004B334E47204B6579E2
:206E0000657200545820310054582032002077706D0050726F6772616D204D656D6F7279BB
:206E200000446F6E6500526570656174204D656D6F727920004D656D6F727920656D707463
:206E4000790050617573650041626F72740053657269616C3A200049616D62696320410063
:206E600049616D626963204200556C74696D6174696300456E7465722053657269616C2021
:206E80002300427567005458204F6666005458204F6E00506164646C652052657665727360
:206EA0006500506164646C65204E6F726D616C0053696465746F6E65204F66660053696404
:206EC00065746F6E65204F6E0054756E650050545420496E766F6B650057504D2041646A77
:206EE000757374004175746F7370616365204F6666004175746F7370616365204F6E005084
:206F0000676D204D656D6F72792000000B0A000A000A000A000A000A000101000301010195
:206F2000FF0101FF8000BD06000000000000BD23CD2B0000400014005400000000006F25FA
:206F40003E25F72400251525262500000000372BCD2BCA2AFE2ADE2A272BFFFFFFFFFFFF3F
:206F6000FFFFFFFFFFFFFFFFFFFFFFFFFFFFFFFFFFFFFFFFFFFFFFFFFFFFFFFFFFFFFFFF31
:206F8000FFFFFFFFFFFFFFFFFFFFFFFFFFFFFFFFFFFFFFFFFFFFFFFFFFFFFFFFFFFFFFFF11
:206FA000FFFFFFFFFFFFFFFFFFFFFFFFFFFFFFFFFFFFFFFFFFFFFFFFFFFFFFFFFFFFFFFFF1
:206FC000FFFFFFFFFFFFFFFFFFFFFFFFFFFFFFFFFFFFFFFFFFFFFFFFFFFFFFFFFFFFFFFFD1
:207800000C94343C0C94513C0C94513C0C94513C0C94513C0C94513C0C94513C0C94513C1D
:207820000C94513C0C94513C0C94513C0C94513C0C94513C0C94513C0C94513C0C94513CE0
:207840000C94513C0C94513C0C94513C0C94513C0C94513C0C94513C0C94513C0C94513CC0
:207860000C94513C0C94513C11241FBECFEFD8E0DEBFCDBF11E0A0E0B1E0ECE9FFE702C07E
:2078800005900D92A230B107D9F712E0A2E0B1E001C01D92AD30B107E1F70E942D3D0C94CC
:2078A000CC3F0C94003C982F9595959595959595905D8F708A307CF0282F295A8091C000B5
:2078C00085FFFCCF9093C6008091C00085FFFCCF2093C6000895282F205DF0CF982F8091CF
:2078E000C00085FFFCCF9093C6000895EF92FF920F931F93EE24FF2487018091C00087FD7B
:2079000017C00894E11CF11C011D111D81E4E81682E4F8068FE0080780E0180770F3E09106
:207920000401F091050109958091C00087FFE9CF8091C6001F910F91FF90EF9008950E949A
:20794000763C982F8091C00085FFFCCF9093C60091362CF490330CF09053892F08959755DB
:20796000892F08951F930E949F3C182F0E949F3C1295107F810F1F9108951F93182F882308
:2079800021F00E94763C1150E1F71F9108951F93182F0E94763C803249F0809103018F5FC1
:2079A000809303018530C1F01F9108958091C00085FFFCCF84E18093C6008091C00085FF4A
:2079C000FCCF1093C6008091C00085FFFCCF80E18093C6001F910895E0910401F0910501CF
:2079E00009951F9108950E94763C803241F0809103018F5F80930301853081F00895809177
:207A0000C00085FFFCCF84E18093C6008091C00085FFFCCF80E18093C6000895E0910401AC
:207A2000F09105010995089540E951E08823A1F02D9A28EE33E0FA013197F1F72150304072
:207A4000D1F72D9828EE33E0FA013197F1F721503040D1F7815061F708953F924F925F92B3
:207A60006F927F928F929F92AF92BF92CF92DF92EF92FF920F931F93CF93DF93000080E1A3
:207A80008093C4001092C50088E18093C10086E08093C2005098589A259A81E00E94143D43
:207AA00024E1F22E9EE1E92E85E9D82E0FE0C02E10E1B12EAA24A394B1E49B2EA6E58A2E44
:207AC000F2E57F2EE0E26E2E79E4572E63E5462E50E5352E0E94763C8033B1F18133B9F187
:207AE000803409F46FC0813409F476C0823409F485C0853409F488C0803531F1823521F128
:207B0000813511F1853509F485C0863509F48DC0843609F496C0843709F403C1853709F46A
:207B200072C1863709F466C0809103018F5F80930301853079F6E0910401F0910501099559
:207B40000E94763C803351F60E94F33CC3CF0E94763C803249F78091C00085FFFCCFF0928C
:207B6000C6008091C00085FFFCCF9092C6008091C00085FFFCCF8092C6008091C00085FFEA
:207B8000FCCF7092C6008091C00085FFFCCF6092C6008091C00085FFFCCF5092C6008091A1
:207BA000C00085FFFCCF4092C6008091C00085FFFCCF3092C6008091C00085FFFCCFB09214
:207BC000C60088CF0E94763C863808F4BDCF0E94763C0E94F33C7ECF0E94763C803809F473
:207BE0009CC0813809F40BC1823809F43CC1883909F48FC080E00E94C73C6CCF84E10E949F
:207C0000BD3C0E94F33C66CF85E00E94BD3C0E94F33C60CF0E94763C809306010E94763CA3
:207C2000809307010E94F33C55CF0E94763C803309F41DC183E00E94BD3C80E00E94C73C4F
:207C400049CF0E94763C809309020E94763C8093080280910C028E7F80930C020E94763C88
:207C6000853409F415C18091080290910902892B89F000E010E00E94763CF801E85FFE4F53
:207C800080830F5F1F4F80910802909109020817190788F30E94763C803209F045CF8091E0
:207CA0000C0280FF01C16091060170910701660F771F7093070160930601A0910802B091E8
:207CC00009021097C9F0E8E0F1E09B01AD014E0F5F1FF999FECF32BD21BD819180BDFA9A6C
:207CE000F99A2F5F3F4FE417F50799F76A0F7B1F70930701609306018091C00085FFFCCF16
:207D0000F092C6008091C00085FFFCCFB092C600E1CE83E00E94C73CDDCE82E00E94C73C8A
:207D2000D9CE0E94763C809309020E94763C809308028091060190910701880F991F909306
:207D40000701809306010E94763C853409F4A6C080910C028E7F80930C020E94763C80323E
:207D600009F0B8CE8091C00085FFFCCFF092C600609108027091090261157105B9F140E05F
:207D800050E080910C02A82FA170B82FB27011C0BB2309F45CC0E0910601F0910701319613
:207DA000F0930701E09306014F5F5F4F46175707E8F4AA2369F3F999FECF209106013091CA
:207DC000070132BD21BDF89A90B58091C00085FFFCCF9093C6002F5F3F4F30930701209354
:207DE00006014F5F5F4F4617570718F38091C00085FDE5CE8091C00085FFF8CFE0CE81E029
:207E00000E94C73C67CE0E94763C803209F08CCE8091C00085FFFCCFF092C6008091C000F6
:207E200085FFFCCFE092C6008091C00085FFFCCFD092C6008091C00085FFFCCFC092C6003B
:207E40008091C00085FFFCCFB092C60043CEE0910601F091070194918091C00085FFFCCFA3
:207E60009093C6009CCF80E10E94C73C33CE0E94763C0E94763C182F0E94763C112309F433
:207E800083C0113009F484C08FE00E94C73C22CE80910C02816080930C02E5CE80910C0226
:207EA000816080930C0259CF809107018823880F880B8A2180930B0280910601909107019E
:207EC000880F991F90930701809306018091080280FF09C0809108029091090201969093AA
:207EE000090280930802F894F999FECF1127E0910601F0910701C8E0D1E0809108029091A1
:207F00000902103091F40091570001700130D9F303E000935700E895009157000170013067
:207F2000D9F301E100935700E895099019900091570001700130D9F301E000935700E8954C
:207F40001395103498F011270091570001700130D9F305E000935700E8950091570001707A
:207F60000130D9F301E100935700E8953296029709F0C7CF103011F00296E5CF11248091F8
:1E7F8000C00085FFB9CEBCCE8EE10E94C73CA2CD85E90E94C73C9ECDF894FFCF8000B3
:00000001FF
